:020000040000FA
:0408000098EF0BF072
:1008100003B275EF05F0F2B493EF05F09EB09BEFD5
:1008200005F09EB2A3EF05F0F2A81AEF04F0F2B2C1
:1008300023EF04F0F2B01FEF04F047EF0BF0F29655
:10084000F29047EF0BF0CD90F2929EA02DEF04F0C6
:100850000101533F2DEF04F0542BB2C1B6F1B3C1E7
:10086000B7F1B4C1B8F1B5C1B9F1AEC1B2F1AFC120
:10087000B3F1B0C1B4F1B1C1B5F1AAC1AEF1ABC130
:10088000AFF1ACC1B0F1ADC1B1F1A6C1AAF1A7C140
:10089000ABF1A8C1ACF1A9C1ADF1A2C1A6F1A3C150
:1008A000A7F1A4C1A8F1A5C1A9F19EC1A2F19FC160
:1008B000A3F1A0C1A4F1A1C1A5F19AC19EF19BC170
:1008C0009FF19CC1A0F19DC1A1F1CECF9AF1CFCFF4
:1008D0009BF153C19CF154C19DF1CF6ACE6A0101D5
:1008E000536B546B9E90CD800FBC0F8E0FBA7CEF74
:1008F00004F00F8A47EF0BF013880F8C0FBEB9EF8F
:1009000004F09AC19EF19BC19FF19CC1A0F19DC1D1
:10091000A1F19EC1A2F19FC1A3F1A0C1A4F1A1C107
:10092000A5F1A2C1A6F1A3C1A7F1A4C1A8F1A5C1D7
:10093000A9F1A6C1AAF1A7C1ABF1A8C1ACF1A9C1A7
:10094000ADF1AAC1AEF1ABC1AFF1ACC1B0F1ADC177
:10095000B1F1AEC1B2F1AFC1B3F1B0C1B4F1B1C147
:10096000B5F1B2C1B6F1B3C1B7F1B4C1B8F1B5C117
:10097000B9F101015E6B5F6B606B616B9A515E2731
:100980009B515F239C5160239D5161239E515E27A3
:100990009F515F23A0516023A1516123A2515E2783
:1009A000A3515F23A4516023A5516123A6515E2763
:1009B000A7515F23A8516023A9516123AA515E2743
:1009C000AB515F23AC516023AD516123AE515E2723
:1009D000AF515F23B0516023B1516123B2515E2703
:1009E000B3515F23B4516023B5516123B6515E27E3
:1009F000B7515F23B8516023B9516123D8900101E9
:100A0000613360335F335E33D8900101613360330B
:100A10005F335E33D8900101613360335F335E33FF
:100A200000C10CF101C10DF102C10EF103C10FF1C2
:100A300004C110F105C111F106C112F107C113F192
:100A400008C114F109C115F10AC116F10BC117F162
:100A500034C135F111B838EF05F00101620E046FB1
:100A6000010E056F000E066F000E076F41EF05F0D7
:100A70000101A70E046F020E056F000E066F000E37
:100A8000076F5EC100F15FC101F160C102F161C198
:100A900003F1FEEC2FF003BF04D01CBE02D01CA05B
:100AA000108C11A059EF05F010BA59EF05F00F8026
:100AB000108A0CC100F10DC101F10EC102F10FC18C
:100AC00003F110C104F111C105F112C106F113C106
:100AD00007F114C108F115C109F116C10AF117C1D6
:100AE0000BF135C134F147EF0BF00392ABB2AB9889
:100AF000AB88030103EE00F080517F0BE92604C0B0
:100B0000EFFF802B8151805D700BD8A48B82000099
:100B10008051815D700BD8A48B9281518019D8B41B
:100B2000079047EF0BF0F2940101453F47EF0BF0C0
:100B3000462B47EF0BF09E900101533F47EF0BF020
:100B4000542B47EF0BF09E9211B843EF08F00400CE
:100B500066A1ABEF05F08BB4B5EF05F010ACB5EFC7
:100B600005F08B84109CB6EF05F08B94077C07ACE6
:100B7000D1EF05F0C274C2B4CBEF05F0C3CFB7F527
:100B8000C4CFB8F50501D890B833B733D890B8338F
:100B9000B733D2EF05F0C3CF55F1C4CF56F1D2EF42
:100BA00005F0C28207B444EF06F047C14BF148C1DB
:100BB0004CF149C14DF14AC14EF15EC162F15FC1D4
:100BC00063F160C164F161C165F113A8EAEF05F05A
:100BD000138C13989AC1BAF19BC1BBF19CC1BCF1B3
:100BE0009DC1BDF19EC1BEF19FC1BFF1A0C1C0F1C9
:100BF000A1C1C1F1A2C1C2F1A3C1C3F1A4C1C4F199
:100C0000A5C1C5F1A6C1C6F1A7C1C7F1A8C1C8F168
:100C1000A9C1C9F1AAC1CAF1ABC1CBF1ACC1CCF138
:100C2000ADC1CDF1AEC1CEF1AFC1CFF1B0C1D0F108
:100C3000B1C1D1F1B2C1D2F1B3C1D3F1B4C1D4F1D8
:100C4000B5C1D5F1B6C1D6F1B7C1D7F1B8C1D8F1A8
:100C5000B9C1D9F1B7C5B9F5B8C5BAF5B9C5BBF5CC
:100C6000BAC5BCF5010155515B2756515C23E86AB2
:100C70005D230E2E44EF06F05CC157F15DC158F1C3
:100C80005B6B5C6B5D6B078E0201002F47EF0BF017
:100C90003C0E006F1D50E00BE00AE86612881BBE98
:100CA00002D01BB4108E00C10CF101C10DF102C1C4
:100CB0000EF103C10FF104C110F105C111F106C11C
:100CC00012F107C113F108C114F109C115F10AC1EC
:100CD00016F10BC117F134C135F181AAACEF06F062
:100CE00015A4F7EF06F005012F51000AD8B43AEF2A
:100CF00007F005012F51010AD8B4B6EF06F005013F
:100D00002F51020AD8B4F7EF06F005012F51030A5C
:100D1000D8B4F7EF06F005012F51040AD8B4F7EF65
:100D200006F005012F51050AD8B4F7EF06F00501CA
:100D30002F51060AD8B4F7EF06F005012F51070A24
:100D4000D8B4F7EF06F005012F51320AD8B4B4EF4A
:100D500006F02F6B3AEF07F000011650030AD8B4E3
:100D6000F7EF06F03AEF07F03AEF07F005015767A3
:100D7000C1EF06F05867C1EF06F05967C1EF06F002
:100D80005A67C5EF06F03AEF07F05BC500F15CC5A6
:100D900001F15DC502F15EC503F10101010E046FB1
:100DA000000E056F000E066F000E076FFEEC2FF0B1
:100DB00000C15BF501C15CF502C15DF503C15EF5E3
:100DC00001010067EBEF06F00167EBEF06F0026749
:100DD000EBEF06F003673AEF07F057C55BF558C530
:100DE0005CF559C55DF55AC55EF524EF07F00FBEF9
:100DF0000CEF07F010A011EF07F00101476708EFB3
:100E000007F0486708EF07F0496708EF07F04A67FF
:100E10000CEF07F011EF07F007AE11EF07F024EF2A
:100E200007F00501312F3AEF07F03C0E316F302FFC
:100E30003AEF07F00101000E626FE00E636FA50E3E
:100E4000646F010E656F138800011650000AD8B454
:100E500032EF07F000011650030AD8B437EF07F05D
:100E60003AEF07F00001010E166E3AEF07F00001AD
:100E7000040E166E0501666B37B740EF07F066810A
:100E80000CC100F10DC101F10EC102F10FC103F15E
:100E900010C104F111C105F112C106F113C107F12E
:100EA00014C108F115C109F116C10AF117C10BF1FE
:100EB00035C134F100C10CF101C10DF102C10EF1D7
:100EC00003C10FF104C110F105C111F106C112F106
:100ED00007C113F108C114F109C115F10AC116F1D6
:100EE0000BC117F134C135F101018E677FEF07F0B7
:100EF0008F677FEF07F090677FEF07F0916783EFD1
:100F000007F0B4EF07F092C100F193C101F194C171
:100F100002F195C103F10101010E046F000E056F8E
:100F2000000E066F000E076FFEEC2FF000C192F16D
:100F300001C193F102C194F103C195F10101006770
:100F4000A9EF07F00167A9EF07F00267A9EF07F023
:100F50000367B4EF07F08EC192F18FC193F190C196
:100F600094F191C195F10F80D57ED5BE6ED0D6CFCC
:100F700047F1D7CF48F145C149F1E86AE8CF4AF1D6
:100F8000138A1CBE02D01CA0108C109047C100F127
:100F900048C101F149C102F14AC103F101010A0E40
:100FA000046F000E056F000E066F000E076FFEEC5B
:100FB0002FF003AF1080010154A7EBEF07F00F9A59
:100FC0000F9C0F9E0101000E5E6F600E5F6F3D0E65
:100FD000606F080E616F010147BFFBEF07F04867C4
:100FE000FBEF07F04967FBEF07F04A67FBEF07F0FD
:100FF000F28820EF08F0F2985E6B5F6B606B616BBC
:101000009A6B9B6B9C6B9D6B9E6B9F6BA06BA16B9C
:10101000A26BA36BA46BA56BA66BA76BA86BA96B4C
:10102000AA6BAB6BAC6BAD6BAE6BAF6BB06BB16BFC
:10103000B26BB36BB46BB56BB66BB76BB86BB96BAC
:10104000D76AD66A0101456B466B0CC100F10DC130
:1010500001F10EC102F10FC103F110C104F111C180
:1010600005F112C106F113C107F114C108F115C150
:1010700009F116C10AF117C10BF135C134F147EF7F
:101080000BF047EF0BF00201002FABEF0AF0D59EFB
:10109000D6CF47F1D7CF48F145C149F1E86AE8CF4B
:1010A0004AF1138AD76AD66A0101456B466BD58E21
:1010B0001D50E00BE00AE86612881BBE02D01BB48C
:1010C000108E1AAE1F8C00C10CF101C10DF102C1CE
:1010D0000EF103C10FF104C110F105C111F106C1F8
:1010E00012F107C113F108C114F109C115F10AC1C8
:1010F00016F10BC117F134C135F10FA0109A11B8D8
:101100008DEF08F00101620E046F010E056F000EF5
:10111000066F000E076F96EF08F00101A70E046F2F
:10112000020E056F000E066F000E076F47C100F13B
:1011300048C101F149C102F14AC103F1FEEC2FF0AF
:1011400003BFA9EF08F01CBE02D01CA0108C11B088
:101150000F800CC100F10DC101F10EC102F10FC1F0
:1011600003F110C104F111C105F112C106F113C15F
:1011700007F114C108F115C109F116C10AF117C12F
:101180000BF135C134F102013C0E006F00C10CF1CE
:1011900001C10DF102C10EF103C10FF104C110F143
:1011A00005C111F106C112F107C113F108C114F113
:1011B00009C115F10AC116F10BC117F134C135F19E
:1011C00081BAE6EF08F015B225EF09F015A025EF7A
:1011D00009F015A470EF09F005012F51000AD8B4E9
:1011E000B3EF09F005012F51010AD8B42FEF09F030
:1011F00005012F51020AD8B470EF09F005012F51F3
:10120000030AD8B470EF09F005012F51040AD8B4CD
:1012100070EF09F005012F51050AD8B470EF09F0FD
:1012200005012F51060AD8B470EF09F005012F51BE
:10123000070AD8B470EF09F005012F51320AD8B46B
:101240002DEF09F02F6BB3EF09F000011650030AE0
:10125000D8B470EF09F0B3EF09F0B3EF09F005016E
:1012600057673AEF09F058673AEF09F059673AEFD4
:1012700009F05A673EEF09F0B3EF09F05BC500F1E2
:101280005CC501F15DC502F15EC503F10101010E0E
:10129000046F000E056F000E066F000E076FFEEC68
:1012A0002FF000C15BF501C15CF502C15DF503C122
:1012B0005EF50101006764EF09F0016764EF09F072
:1012C000026764EF09F00367B3EF09F057C55BF5F8
:1012D00058C55CF559C55DF55AC55EF59DEF09F039
:1012E0000FBE85EF09F010A08AEF09F001014767F2
:1012F00081EF09F0486781EF09F0496781EF09F054
:101300004A6785EF09F08AEF09F007AE8AEF09F026
:101310009DEF09F00501312FB3EF09F03C0E316F5D
:10132000302FB3EF09F00101000E626FE00E636F22
:10133000A50E646F010E656F138800011650000A38
:10134000D8B4ABEF09F000011650030AD8B4B0EFDF
:1013500009F0B3EF09F00001010E166EB3EF09F0CA
:101360000001040E166E0501666B37B7B9EF09F080
:1013700066810CC100F10DC101F10EC102F10FC176
:1013800003F110C104F111C105F112C106F113C13D
:1013900007F114C108F115C109F116C10AF117C10D
:1013A0000BF135C134F100C10CF101C10DF102C1E5
:1013B0000EF103C10FF104C110F105C111F106C115
:1013C00012F107C113F108C114F109C115F10AC1E5
:1013D00016F10BC117F134C135F101018E67F8EF39
:1013E00009F08F67F8EF09F09067F8EF09F091675F
:1013F000FCEF09F02DEF0AF092C100F193C101F169
:1014000094C102F195C103F10101010E046F000EB8
:10141000056F000E066F000E076FFEEC2FF000C187
:1014200092F101C193F102C194F103C195F101015F
:10143000006722EF0AF0016722EF0AF0026722EF4D
:101440000AF003672DEF0AF08EC192F18FC193F17C
:1014500090C194F191C195F10F80109047C100F1B6
:1014600048C101F149C102F14AC103F101010A0E6B
:10147000046F000E056F000E066F000E076FFEEC86
:101480002FF003AF1080010154A753EF0AF00F9A19
:101490000F9C0F9E0101000E5E6F600E5F6F3D0E90
:1014A000606F080E616F47C100F148C101F149C189
:1014B00002F14AC103F10101140E046F050E056F1C
:1014C000000E066F000E076FFEEC2FF003AF6CEFFF
:1014D0000AF0F28891EF0AF0F2985E6B5F6B606B36
:1014E000616B9A6B9B6B9C6B9D6B9E6B9F6BA06BF8
:1014F000A16BA26BA36BA46BA56BA66BA76BA86B70
:10150000A96BAA6BAB6BAC6BAD6BAE6BAF6BB06B1F
:10151000B16BB26BB36BB46BB56BB66BB76BB86BCF
:10152000B96B0CC100F10DC101F10EC102F10FC187
:1015300003F110C104F111C105F112C106F113C18B
:1015400007F114C108F115C109F116C10AF117C15B
:101550000BF135C134F104008BB4B6EF0AF010ACD6
:10156000B6EF0AF08B84109CB7EF0AF08B94077CDF
:1015700007ACD2EF0AF0C274C2B4CCEF0AF0C3CF0A
:10158000B7F5C4CFB8F50501D890B833B733D890C4
:10159000B833B733D3EF0AF0C3CF55F1C4CF56F108
:1015A000D3EF0AF0C28207B445EF0BF047C14BF10D
:1015B00048C14CF149C14DF14AC14EF15EC162F1E1
:1015C0005FC163F160C164F161C165F113A8EBEF24
:1015D0000AF0138C13989AC1BAF19BC1BBF19CC15C
:1015E000BCF19DC1BDF19EC1BEF19FC1BFF1A0C1C3
:1015F000C0F1A1C1C1F1A2C1C2F1A3C1C3F1A4C193
:10160000C4F1A5C1C5F1A6C1C6F1A7C1C7F1A8C162
:10161000C8F1A9C1C9F1AAC1CAF1ABC1CBF1ACC132
:10162000CCF1ADC1CDF1AEC1CEF1AFC1CFF1B0C102
:10163000D0F1B1C1D1F1B2C1D2F1B3C1D3F1B4C1D2
:10164000D4F1B5C1D5F1B6C1D6F1B7C1D7F1B8C1A2
:10165000D8F1B9C1D9F1B7C5B9F5B8C5BAF5B9C5A9
:10166000BBF5BAC5BCF5010155515B2756515C234A
:10167000E86A5D230E2E45EF0BF05CC157F15DC1AA
:1016800058F15B6B5C6B5D6B078E47EF0BF002C034
:10169000E0FF005001C0D8FF1000A6B24DEF0BF0E4
:1016A0000CC0A9FF0BC0A8FFA69EA69CA684F29E14
:1016B000550EA76EAA0EA76EA682F28EA694A6B2AB
:1016C0005FEF0BF00C2A1200A96EA69EA69CA680C6
:1016D000A8500C2A120004012C0E826F94EC0EF01C
:1016E00013EC31F00C5064EC0BF0E8CF00F10C502F
:1016F00064EC0BF0E8CF01F101AF84EF0BF00101D6
:10170000FF0E026FFF0E036F9CEC30F0296790EF25
:101710000BF00401200E826F94EC0EF095EF0BF0AD
:1017200004012D0E826F94EC0EF0A6EC2EF0120048
:1017300015941596076A0F6A106A116A126A136A7D
:10174000166A0F010D0EC16E860EC06E030EC26EBC
:101750000F01680E896E130E926E080E8A6EF30EDC
:10176000936E8B6A900E946EC80E64EC0BF0E8CF0B
:10177000E8FF1098E8A0108810A805D00E0E256E7E
:101780008E0E266E04D00F0E256E8F0E266EABECDD
:1017900031F0F18EF19EFC0E64EC0BF0E8CF0BF013
:1017A0000BA011800BA211820BA411840BA811882D
:1017B000C90E64EC0BF0E8CF1AF0CA0E64EC0BF023
:1017C000E8CF1BF0CB0E64EC0BF0E8CF1CF0CC0E96
:1017D00064EC0BF0E8CF1DF0FB0E64EC0BF0E8CFEF
:1017E00037F0CE0E64EC0BF0E8CF14F0CD0E64ECC5
:1017F0000BF0E8CF36F01F6A206A0E6A01015B6BBE
:101800005C6B5D6B576B586BF29A0101476B486BD1
:10181000496B4A6B4B6B4C6B4D6B4E6B4F6B506B0C
:10182000516B526B456B466BD76AD66A0F01280E17
:10183000D56EF28A9D90B00ECD6E01015E6B5F6B2E
:10184000606B616B626B636B646B656B666B676B24
:10185000686B696B536B546BCF6ACE6A0F9A0F9C9F
:101860000F9E9D80760ECA6E9D8202013C0E006F17
:10187000CC6A160E64EC0BF0E8CF00F1170E64ECA6
:101880000BF0E8CF01F1180E64EC0BF0E8CF02F199
:10189000190E64EC0BF0E8CF03F1010103AF6BEF1D
:1018A0000CF013EC31F0160E0C6E00C10BF04DEC89
:1018B0000BF0170E0C6E01C10BF04DEC0BF0180E77
:1018C0000C6E02C10BF04DEC0BF0190E0C6E03C147
:1018D0000BF04DEC0BF000C18EF101C18FF102C194
:1018E00090F103C191F100C192F101C193F102C1E4
:1018F00094F103C195F11A0E64EC0BF0E8CF00F1FE
:101900001B0E64EC0BF0E8CF01F11C0E64EC0BF045
:10191000E8CF02F11D0E64EC0BF0E8CF03F10101FA
:1019200003AFC1EF0CF013EC31F01A0E0C6E00C1D6
:101930000BF04DEC0BF01B0E0C6E01C10BF04DECDF
:101940000BF01C0E0C6E02C10BF04DEC0BF01D0EDB
:101950000C6E03C10BF04DEC0BF01A0E64EC0BF0A7
:10196000E8CF00F11B0E64EC0BF0E8CF01F11C0E88
:1019700064EC0BF0E8CF02F11D0E64EC0BF0E8CF45
:1019800003F100C196F101C197F102C198F103C1C1
:1019900099F1240EAC6E900EAB6E240EAC6E080E58
:1019A000B86E000EB06E1F0EAF6E0401806B816BBF
:1019B0000F01900EAB6E0F019D8A0301806B816B4E
:1019C000C26B8B9250EC36F050EC36F032EC38F0C3
:1019D0002EEC34F0200E64EC0BF0E8CF2FF505016F
:1019E0002F51FF0AD8A4FCEF0CF02F6B200E0C6EC9
:1019F0002FC50BF04DEC0BF00501010E306F3C0EC6
:101A0000316F250E64EC0BF0E8CF00F1260E64EC8C
:101A10000BF0E8CF01F1270E64EC0BF0E8CF02F1F8
:101A2000280E64EC0BF0E8CF03F1010103AF33EFB4
:101A30000DF013EC31F0250E0C6E00C10BF04DECE7
:101A40000BF0260E0C6E01C10BF04DEC0BF0270EC7
:101A50000C6E02C10BF04DEC0BF0280E0C6E03C1A6
:101A60000BF04DEC0BF000C157F501C158F502C168
:101A700059F503C15AF500C15BF501C15CF502C11E
:101A80005DF503C15EF5290E64EC0BF0E8CF5FF560
:101A9000050160515F5DD8A05FC560F5210E64EC63
:101AA0000BF0E8CF00F1220E64EC0BF0E8CF01F16F
:101AB000230E64EC0BF0E8CF02F1240E64EC0BF083
:101AC000E8CF03F1010103AF94EF0DF013EC31F017
:101AD000210E0C6E00C10BF04DEC0BF0220E0C6EC3
:101AE00001C10BF04DEC0BF0230E0C6E02C10BF09C
:101AF0004DEC0BF0240E0C6E03C10BF04DEC0BF013
:101B0000210E64EC0BF0E8CF00F1220E64EC0BF038
:101B1000E8CF01F1230E64EC0BF0E8CF02F1240EC4
:101B200064EC0BF0E8CF03F100C161F501C162F58F
:101B300002C163F503C164F576EC33F05CEC32F07E
:101B4000B4EC31F01590C70E64EC0BF0E8CF00F167
:101B5000010100B1AFEF0DF01592B0EF0DF015825D
:101B600081AABEEF0DF015B4B9EF0DF01580BEEFF0
:101B70000DF071EC38F015A0D8EF38F007900001A7
:101B8000F28EF28C12AE03D012BC6CEF19F007B0DB
:101B900025EF2DF00FB021EF26F010BE21EF26F03B
:101BA00012B821EF26F000011650010AD8B41AEF3E
:101BB0001EF081BAE4EF0DF000011650040AD8B40B
:101BC00018EF1CF0EAEF0DF000011650040AD8B42B
:101BD00056EF1EF00301805181197F0BD8B425EF19
:101BE0002DF013EE00F081517F0BE126812BE7CF22
:101BF000E8FFE00BD8B425EF2DF023EE82F0C251C0
:101C00003F0BD926E7CFDFFFC22BDF50780AD8A4DD
:101C100025EF2DF0078092C100F193C101F194C12D
:101C200002F195C103F10101040E046F000E056F6E
:101C3000000E066F000E076FFEEC2FF000AF2AEFCC
:101C40000EF00101030E926F000E936F000E946F61
:101C5000000E956F03018251720AD8B4A2EF25F0ED
:101C60008251520AD8B4A2EF25F08251750AD8B435
:101C7000A2EF25F08251680AD8B4A8EF0EF0825185
:101C8000630AD8B4DFEF29F08251690AD8B460EF53
:101C900021F082517A0AD8B473EF22F08251490AB6
:101CA000D8B4FFEF20F08251500AD8B41DEF20F0D5
:101CB0008251700AD8B460EF20F08251540AD8B42F
:101CC0008BEF20F08251740AD8B4D1EF20F082510A
:101CD000410AD8B4ADEF0FF082514B0AD8B4AAEF45
:101CE0000EF082516D0AD8B41DEF14F082514D0AE6
:101CF000D8B436EF14F08251730AD8B4D2EF24F07E
:101D00008251530AD8B437EF25F082514C0AD8B427
:101D1000C5EF14F08251590AD8B46EEF13F012AE29
:101D200001D0128C16EF2AF0040114EE00F080515D
:101D30007F0BE12682C4E7FF802B120004010D0E09
:101D4000826F94EC0EF00A0E826F94EC0EF012008B
:101D500014EF2AF004014B0E826F94EC0EF0040194
:101D60002C0E826F94EC0EF081B802D036B630D0D3
:101D700003018351430AD8B4EFEF0EF003018351FE
:101D8000630AD8B4F1EF0EF003018351520AD8B4BC
:101D9000F3EF0EF003018351720AD8B4F5EF0EF0A1
:101DA00003018351470AD8B4F7EF0EF003018351C2
:101DB000670AD8B4F9EF0EF003018351540AD8B47E
:101DC000FBEF0EF003018351740AD8B46BEF0FF0F0
:101DD00003018351550AD8B4FDEF0EF083D036804D
:101DE0007BD0369079D0368277D0369275D03684D3
:101DF00073D0369471D036866FD084C330F185C3EA
:101E000031F186C332F187C333F10101296B61ECF3
:101E100031F0D8EC30F000C104F101C105F102C18C
:101E200006F103C107F154EC31F0200EF86EF76AA9
:101E3000F66A0900F5CF2CF10900F5CF2DF1090064
:101E4000F5CF2EF10900F5CF2FF10900F5CF30F1D4
:101E50000900F5CF31F10900F5CF32F10900F5CFD6
:101E600033F10101296B61EC31F0D8EC30F0FEEC7C
:101E70002FF00101006744EF0FF0016744EF0FF00E
:101E8000026744EF0FF0036701D025D004014E0E26
:101E9000826F94EC0EF004016F0E826F94EC0EF0E2
:101EA00004014D0E826F94EC0EF00401610E826FFE
:101EB00094EC0EF00401740E826F94EC0EF00401A9
:101EC000630E826F94EC0EF00401680E826F94EC46
:101ED0000EF014EF2AF03696CD0E0C6E36C00BF0D5
:101EE0004DEC0BF0CD0E64EC0BF0E8CF36F036B0D5
:101EF00006D00401630E826F94EC0EF005D004014D
:101F0000430E826F94EC0EF036B206D00401720ECE
:101F1000826F94EC0EF005D00401520E826F94ECA7
:101F20000EF036B406D00401670E826F94EC0EF00A
:101F300005D00401470E826F94EC0EF036B606D041
:101F40000401740E826F94EC0EF005D00401540E5F
:101F5000826F94EC0EF014EF2AF00401410E826FB0
:101F600094EC0EF003018351310AD8B48EEF12F0D5
:101F700003018351320AD8B4BEEF11F0030183513B
:101F8000330AD8B447EF11F003018351340AD8B4AF
:101F900037EF10F003018351350AD8B4D7EF0FF0B3
:101FA00004013F0E826F94EC0EF014EF2AF003014F
:101FB0008451300AD8B4FDEF0FF003018451310A87
:101FC000D8B400EF10F003018451650AD8B4F1EFE2
:101FD0000FF003018451640AD8B4F4EF0FF001EF5D
:101FE00010F03790F5EF0FF03780FB0E0C6E37C016
:101FF0000BF04DEC0BF001EF10F08B9001EF10F0B7
:102000008B800401350E826F94EC0EF004012C0ECF
:10201000826F94EC0EF08BB015EF10F00401300ECF
:10202000826F94EC0EF01AEF10F00401310E826F03
:1020300094EC0EF004012C0E826F94EC0EF0FB0E6B
:1020400064EC0BF0E8CF37F037A02EEF10F004016E
:10205000640E826F94EC0EF033EF10F00401650E05
:10206000826F94EC0EF035EF10F014EF2AF0CC0EE6
:1020700064EC0BF0E8CF0BF004012C0E826F94ECB3
:102080000EF003018451310AD8B45BEF10F0030164
:102090008451300AD8B45DEF10F0030184514D0A29
:1020A000D8B467EF10F003018451540AD8B46EEF2E
:1020B00010F085EF10F08A8401D08A940BAE04D022
:1020C0000BAC02D00BBA21D0E00E0B1218D01F0EB1
:1020D0000B168539E844E00B0B1211D0E00E0B16FD
:1020E00054EC31F085C332F186C333F10101296B21
:1020F00061EC31F0D8EC30F000511F0B0B12CC0E1C
:102100000C6E0BC00BF04DEC0BF00401340E826F23
:1021100094EC0EF004012C0E826F94EC0EF0CC0EB9
:1021200064EC0BF0E8CF1DF08AB406D00401300E49
:10213000826F94EC0EF005D00401310E826F94ECA6
:102140000EF004012C0E826F94EC0EF01D38E84066
:10215000070BE8CF82F40401300E822794EC0EF0D6
:1021600004012C0E826F94EC0EF013EC31F01D5034
:102170001F0BE8CF00F19CEC30F032C182F4040177
:10218000300E822794EC0EF033C182F40401300E3D
:10219000822794EC0EF004012C0E826F94EC0EF06A
:1021A00013EC31F030C000F100AF0BD0FF0E016F27
:1021B000FF0E026FFF0E036F04012D0E826F94EC71
:1021C0000EF09CEC30F031C182F40401300E822715
:1021D00094EC0EF032C182F40401300E822794ECAC
:1021E0000EF033C182F40401300E822794EC0EF01D
:1021F00004012C0E826F94EC0EF013EC31F02FC022
:1022000000F19CEC30F031C182F40401300E8227E1
:1022100094EC0EF032C182F40401300E822794EC6B
:102220000EF033C182F40401300E822794EC0EF0DC
:1022300004012C0E826F94EC0EF013EC31F031C0DF
:1022400000F100AF0BD0FF0E016FFF0E026FFF0E0B
:10225000036F04012D0E826F94EC0EF09CEC30F0B5
:1022600031C182F40401300E822794EC0EF032C1A9
:1022700082F40401300E822794EC0EF033C182F414
:102280000401300E822794EC0EF014EF2AF0CB0EEE
:1022900064EC0BF0E8CF0BF004012C0E826F94EC91
:1022A0000EF003018451450AD8B46BEF11F003011D
:1022B0008451440AD8B46EEF11F003018451300AFE
:1022C000D8B471EF11F003018451310AD8B475EF1D
:1022D00011F080EF11F00B9E7AEF11F00B8E7AEF78
:1022E00011F0FC0E0B167AEF11F0FC0E0B160B80A2
:1022F0007AEF11F0CB0E0C6E0BC00BF04DEC0BF027
:102300000401330E826F94EC0EF004012C0E826FE8
:1023100094EC0EF0CB0E64EC0BF0E8CF1CF01CBE7E
:1023200099EF11F00401450E826F94EC0EF09EEFD0
:1023300011F00401440E826F94EC0EF004012C0E97
:10234000826F94EC0EF00401300E826F94EC0EF06C
:1023500004012C0E826F94EC0EF01CB0B7EF11F05C
:102360000401300E826F94EC0EF0BCEF11F004010A
:10237000310E826F94EC0EF014EF2AF0CA0E64EC6A
:102380000BF0E8CF0BF004012C0E826F94EC0EF0F2
:1023900003018451450AD8B4FAEF11F003018451C6
:1023A000440AD8B4FDEF11F0030184514D0AD8B4AA
:1023B00006EF12F003018451410AD8B400EF12F085
:1023C00003018451460AD8B403EF12F0030184518B
:1023D000560AD8B40EEF12F003018451500AD8B453
:1023E00019EF12F003018451520AD8B41CEF12F015
:1023F00025EF12F00B9E1FEF12F00B8E1FEF12F065
:102400000B9C1FEF12F00B8C1FEF12F0FC0E0B1643
:1024100085C3E8FF030B0B121FEF12F0C70E0B165C
:1024200085C3E8FF070BE846E846E8460B121FEFB6
:1024300012F00B841FEF12F00B941FEF12F0CA0E74
:102440000C6E0BC00BF04DEC0BF0CA0E64EC0BF0F5
:10245000E8CF1BF00401320E826F94EC0EF0040101
:102460002C0E826F94EC0EF01BBE3EEF12F00401B6
:10247000450E826F94EC0EF043EF12F00401440E0F
:10248000826F94EC0EF004012C0E826F94EC0EF02F
:102490001BC0E8FF030BE8CF82F40401300E822753
:1024A00094EC0EF004012C0E826F94EC0EF01BBC29
:1024B00061EF12F00401410E826F94EC0EF066EFB2
:1024C00012F00401460E826F94EC0EF004012C0E03
:1024D000826F94EC0EF01BC0E8FF380BE842E84234
:1024E000E842E8CF82F40401300E822794EC0EF02B
:1024F00004012C0E826F94EC0EF01BB487EF12F0E7
:102500000401520E826F94EC0EF08CEF12F0040175
:10251000500E826F94EC0EF014EF2AF0C90E64ECAA
:102520000BF0E8CF0BF004012C0E826F94EC0EF050
:1025300003018451450AD8B4ACEF12F00301845171
:10254000440AD8B4AFEF12F0030184514D0AD8B455
:10255000B2EF12F0C0EF12F00B9EBAEF12F00B8E3A
:10256000BAEF12F0F80E0B1685C3E8FF070B0B123B
:10257000BAEF12F0C90E0C6E0BC00BF04DEC0BF065
:102580000401310E826F94EC0EF004012C0E826F68
:1025900094EC0EF0C90E64EC0BF0E8CF1AF01ABE02
:1025A00006D00401450E826F94EC0EF005D00401B4
:1025B000440E826F94EC0EF004012C0E826F94ECAA
:1025C0000EF01AC0E8FF070BE8CF82F40401300ECA
:1025D000822794EC0EF004012C0E826F94EC0EF026
:1025E000078013EC31F02BC0E8FF003B00430043B1
:1025F000030B9CEC30F033C182F40401300E8227CF
:1026000094EC0EF004012C0E826F94EC0EF013EC9F
:1026100031F02BC001F1019F019D2CC000F101019F
:102620009CEC30F02FC182F40401300E822794EC30
:102630000EF030C182F40401300E822794EC0EF0CB
:1026400031C182F40401300E822794EC0EF032C1C5
:1026500082F40401300E822794EC0EF033C182F430
:102660000401300E822794EC0EF004012C0E826FD0
:1026700094EC0EF013EC31F02DC001F12EC000F1FE
:10268000D89001330033D8900133003301019CEC22
:1026900030F02FC182F40401300E822794EC0EF04A
:1026A00030C182F40401300E822794EC0EF031C167
:1026B00082F40401300E822794EC0EF032C182F4D1
:1026C0000401300E822794EC0EF033C182F4040131
:1026D000300E822794EC0EF014EF2AF0FC0E64EC1E
:1026E0000BF0E8CF0BF003018351520AD8B4A5EFE9
:1026F00013F003018351720AD8B4A8EF13F0030159
:102700008351500AD8B4ABEF13F003018351700A20
:10271000D8B4AEEF13F003018351550AD8B4B1EF2A
:1027200013F003018351750AD8B4B4EF13F0030119
:102730008351430AD8B4BDEF13F003018351630AF8
:10274000D8B4C0EF13F0C9EF13F00B90C3EF13F040
:102750000B80C3EF13F00B92C3EF13F00B82C3EFA8
:1027600013F00B94C3EF13F00B84C3EF13F00B962D
:10277000C3EF13F00B86C3EF13F00B98C3EF13F006
:102780000B88C3EF13F0FC0E0C6E0BC00BF04DEC7E
:102790000BF00401590E826F94EC0EF0119011921F
:1027A00011941198FC0E64EC0BF0E8CF0BF00BA029
:1027B00011800BA211820BA411840BA8118811A007
:1027C000E9EF13F00401520E826F94EC0EF0EEEF7D
:1027D00013F00401720E826F94EC0EF011A8F8EF62
:1027E00013F00401430E826F94EC0EF0FDEF13F032
:1027F0000401630E826F94EC0EF011A207EF14F047
:102800000401500E826F94EC0EF00CEF14F00401F2
:10281000700E826F94EC0EF011A416EF14F0040108
:10282000550E826F94EC0EF01BEF14F00401750E40
:10283000826F94EC0EF014EF2AF004016D0E826F9B
:1028400094EC0EF003018351300AD8B475EF14F004
:1028500003018351310AD8B488EF14F00301835186
:10286000320AD8B49BEF14F016EF2AF004014D0E93
:10287000826F94EC0EF054EC31F084C331F185C3D7
:1028800032F186C333F10101296B61EC31F0D8ECF0
:1028900030F003018351300AD8B45DEF14F0030126
:1028A0008351310AD8B465EF14F003018351320A21
:1028B000D8B46DEF14F016EF2AF0FD0E0C6E00C1C7
:1028C0000BF04DEC0BF075EF14F0FE0E0C6E00C12A
:1028D0000BF04DEC0BF088EF14F0FF0E0C6E00C106
:1028E0000BF04DEC0BF09BEF14F00401300E826FF7
:1028F00094EC0EF004012C0E826F94EC0EF013ECAD
:1029000031F0FD0E64EC0BF0E8CF00F1ACEF14F009
:102910000401310E826F94EC0EF004012C0E826FD4
:1029200094EC0EF013EC31F0FE0E64EC0BF0E8CFFB
:1029300000F1ACEF14F00401320E826F94EC0EF053
:1029400013EC31F004012C0E826F94EC0EF0FF0EAC
:1029500064EC0BF0E8CF00F19CEC30F031C182F474
:102960000401300E822794EC0EF032C182F404018F
:10297000300E822794EC0EF033C182F40401300E45
:10298000822794EC0EF014EF2AF003018351300AF1
:10299000D8B419EF1AF003018351310AD8B446EFC5
:1029A0001BF003018351320AD8B4B4EF1BF00301CA
:1029B0008351330AD8B4C4EF1BF003018351340AA6
:1029C000D8B41FEF1CF003018351350AD8B46EEF61
:1029D0001EF003018351360AD8B49CEF1EF00301A8
:1029E0008351370AD8B4F1EF17F003018351380A45
:1029F000D8B48FEF18F003018351440AD8B41DEF07
:102A000016F003018351640AD8B43DEF16F00301B8
:102A10008351460AD8B473EF1DF0030183514D0A68
:102A2000D8B46AEF16F0030183516D0AD8B484EF6D
:102A300016F0030183515A0AD8B4C0EF1AF003010B
:102A40008351490AD8B49CEF1FF003018351500A07
:102A5000D8B4CEEF1EF003018351540AD8B447EF27
:102A60001FF003018351630AD8B4A4EF16F00301E9
:102A70008351430AD8B49CEF17F003018351730AC2
:102A8000D8B4A2EF16F003018351610AD8B46AEFFB
:102A900015F003018351650AD8B469EF1AF00301F8
:102AA0008351450AD8B477EF1AF003018351620AC3
:102AB000D8B485EF1AF003018351420AD8B493EFDA
:102AC0001AF003018351760AD8B4A1EF1AF0D8A402
:102AD00016EF2AF004014C0E826F94EC0EF0040104
:102AE000610E826F94EC0EF05CEC32F004012C0E5F
:102AF000826F94EC0EF013EC31F0AFC500F10101E0
:102B00009CEC30F031C182F40401300E822794EC49
:102B10000EF032C182F40401300E822794EC0EF0E4
:102B200033C182F40401300E822794EC0EF00401CC
:102B30002C0E826F94EC0EF013EC31F0B0C500F166
:102B400001019CEC30F031C182F40401300E822787
:102B500094EC0EF032C182F40401300E822794EC22
:102B60000EF033C182F40401300E822794EC0EF093
:102B700004012C0E826F94EC0EF013EC31F0B1C511
:102B800000F101019CEC30F031C182F40401300EFF
:102B9000822794EC0EF032C182F40401300E8227B9
:102BA00094EC0EF033C182F40401300E822794ECD1
:102BB0000EF004012C0E826F94EC0EF013EC31F049
:102BC000B2C500F101019CEC30F031C182F4040186
:102BD000300E822794EC0EF032C182F40401300EE4
:102BE000822794EC0EF033C182F40401300E822768
:102BF00094EC0EF004012C0E826F94EC0EF013ECAA
:102C000031F0B6C500F101019CEC30F031C182F425
:102C10000401300E822794EC0EF032C182F40401DC
:102C2000300E822794EC0EF033C182F40401300E92
:102C3000822794EC0EF0CAEF1EF003018451300A93
:102C4000D8B429EF16F003018451310AD8B42DEF1E
:102C500016F0159215962EEF16F01582C70E64EC3D
:102C60000BF0E8CF00F10101008115A20091C70E21
:102C70000C6E00C10BF04DEC0BF0C70E64EC0BF0CA
:102C8000E8CF00F1010100B149EF16F015924AEFCB
:102C900016F0158204014C0E826F94EC0EF00401C4
:102CA000640E826F94EC0EF004012C0E826F94EC93
:102CB0000EF015B263EF16F00401300E826F94EC43
:102CC0000EF068EF16F00401310E826F94EC0EF0F6
:102CD00014EF2AF054EC31F084C333F161EC31F09D
:102CE000D8EC30F0200E0C6E00C10BF04DEC0BF068
:102CF00000C12FF505012F51000A06E005012F51F3
:102D0000010A02E0F6EC32F004014C0E826F94EC02
:102D10000EF004014D0E826F94EC0EF004012C0EA7
:102D2000826F94EC0EF013EC31F02FC500F19CECA7
:102D300030F033C182F40401300E822794EC0EF09F
:102D4000CAEF1EF0D8EF38F004014C0E826F94ECFD
:102D50000EF00401630E826F94EC0EF0B4EC31F0CF
:102D600004012C0E826F94EC0EF0B9EC16F0CAEF51
:102D70001EF013EC31F0B5C500F10101003B0F0E60
:102D800000179CEC30F033C182F40401300E82272E
:102D900094EC0EF0B5C500F101010F0E0101001712
:102DA0009CEC30F033C182F40401300E822794ECA5
:102DB0000EF004012D0E826F94EC0EF0B4C500F1FC
:102DC0000101003B0F0E00179CEC30F033C182F480
:102DD0000401300E822794EC0EF0B4C500F101011D
:102DE0000F0E010100179CEC30F033C182F4040196
:102DF000300E822794EC0EF004012D0E826F94ECBD
:102E00000EF0B3C500F10101003B0F0E00179CEC62
:102E100030F033C182F40401300E822794EC0EF0BE
:102E2000B3C500F101010F0E010100179CEC30F059
:102E300033C182F40401300E822794EC0EF00401B9
:102E4000200E826F94EC0EF0B2C500F10F0E01015E
:102E500000179CEC30F033C182F40401300E82275D
:102E600094EC0EF00401200E826F94EC0EF0B1C5CC
:102E700000F101010101003B0F0E00179CEC30F046
:102E800033C182F40401300E822794EC0EF0B1C5F8
:102E900000F101010F0E010100179CEC30F033C16D
:102EA00082F40401300E822794EC0EF004013A0EF5
:102EB000826F94EC0EF0B0C500F10101003B0F0EE3
:102EC00000179CEC30F033C182F40401300E8227ED
:102ED00094EC0EF0B0C500F101010F0E01010017D6
:102EE0009CEC30F033C182F40401300E822794EC64
:102EF0000EF004013A0E826F94EC0EF0AFC500F1B3
:102F00000101003B0F0E00179CEC30F033C182F43E
:102F10000401300E822794EC0EF0AFC500F10101E0
:102F20000F0E00179CEC30F033C182F40401300E18
:102F3000822794EC0EF0120084C3E8FF0F0BE83AEE
:102F4000E8CFB5F585C3E8FF0F0B0501B51387C3BF
:102F5000E8FF0F0BE83AE8CFB4F588C3E8FF0F0BA2
:102F60000501B4138AC3E8FF0F0BE83AE8CFB3F5C5
:102F70008BC3E8FF0F0B0501B3138DC3E8FF0F0BE5
:102F8000E8CFB2F58FC3E8FF0F0BE83AE8CFB1F511
:102F900090C3E8FF0F0B0501B11392C3E8FF0F0BBD
:102FA000E83AE8CFB0F593C3E8FF0F0B0501B01383
:102FB00095C3E8FF0F0BE83AE8CFAFF596C3E8FFFB
:102FC0000F0B0501AF130FEC32F004014C0E826FB2
:102FD00094EC0EF00401430E826F94EC0EF0AEEF11
:102FE00016F0078404014C0E826F94EC0EF004017D
:102FF000370E826F94EC0EF004012C0E826F94EC6D
:103000000EF005012E51130A06E005012E51170A94
:103010000DE08CEF18F00101000E006F000E016F43
:10302000100E026F000E036F1FEF18F00101000E6B
:10303000006F000E016F000E026F010E036F9CEC1B
:1030400030F02AC182F40401300E822794EC0EF095
:103050002BC182F40401300E822794EC0EF02CC1B7
:1030600082F40401300E822794EC0EF02DC182F41C
:103070000401300E822794EC0EF02EC182F404017C
:10308000300E822794EC0EF02FC182F40401300E32
:10309000822794EC0EF030C182F40401300E8227B6
:1030A00094EC0EF031C182F40401300E822794ECCE
:1030B0000EF032C182F40401300E822794EC0EF03F
:1030C00033C182F40401300E822794EC0EF0040127
:1030D0002C0E826F94EC0EF00101200E006F000E9A
:1030E000016F000E026F000E036F9CEC30F031C1D7
:1030F00082F40401300E822794EC0EF032C182F487
:103100000401300E822794EC0EF033C182F40401E6
:10311000300E822794EC0EF00794CAEF1EF00501E2
:10312000216B226B236B246B04014C0E826F94EC99
:103130000EF00401380E826F94EC0EF004012C0E98
:10314000826F94EC0EF00101200E006F000E016FF3
:10315000000E026F000E036F9CEC30F02AC182F467
:103160000401300E822794EC0EF02BC182F404018E
:10317000300E822794EC0EF02CC182F40401300E44
:10318000822794EC0EF02DC182F40401300E8227C8
:1031900094EC0EF02EC182F40401300E822794ECE0
:1031A0000EF02FC182F40401300E822794EC0EF051
:1031B00030C182F40401300E822794EC0EF031C14C
:1031C00082F40401300E822794EC0EF032C182F4B6
:1031D0000401300E822794EC0EF033C182F4040116
:1031E000300E822794EC0EF004012C0E826F94ECCA
:1031F0000EF025C500F126C501F127C502F128C54D
:1032000003F10101200E046F000E056F000E066F22
:10321000000E076F2FEC30F000C133F501C134F51B
:1032200002C135F503C136F59CEC30F02AC182F4B9
:103230000401300E822794EC0EF02BC182F40401BD
:10324000300E822794EC0EF02CC182F40401300E73
:10325000822794EC0EF02DC182F40401300E8227F7
:1032600094EC0EF02EC182F40401300E822794EC0F
:103270000EF02FC182F40401300E822794EC0EF080
:1032800030C182F40401300E822794EC0EF031C17B
:1032900082F40401300E822794EC0EF032C182F4E5
:1032A0000401300E822794EC0EF033C182F4040145
:1032B000300E822794EC0EF09EEC0EF00501336781
:1032C00069EF19F0346769EF19F0356769EF19F0A4
:1032D000366702D008EF1AF0129E129C21C500F149
:1032E00022C501F123C502F124C503F1899A400EDC
:1032F000C76E200EC66E9E96C69E0B0EC96EFF0E42
:103300009EB602D0E82EFCD79E96C69E02C1C9FF8B
:10331000FF0E9EB602D0E82EFCD79E96C69E01C137
:10332000C9FFFF0E9EB602D0E82EFCD79E96C69E21
:1033300000C1C9FFFF0E9EB602D0E82EFCD79E96B4
:10334000C69EC952FF0E9EB602D0E82EFCD70501DC
:10335000200E326F040114EE00F080517F0BE12645
:103360009E96C69EC952FF0E9EB602D0E82EFCD78E
:10337000C9CFE7FF0401802B0501322FAAEF19F016
:10338000898A33C500F134C501F135C502F136C56E
:1033900003F10101010E046F000E056F000E066FB0
:1033A000000E076FFEEC2FF000C133F501C134F5BC
:1033B00002C135F503C136F505013367E7EF19F0B2
:1033C0003467E7EF19F03567E7EF19F0366702D099
:1033D00008EF1AF021C500F122C501F123C502F161
:1033E00024C503F10101200E046F000E056F000ECD
:1033F000066F000E076F03EC30F000C121F501C12C
:1034000022F502C123F503C124F5128E16EF2AF02E
:103410000401450E826F94EC0EF004014F0E826F92
:1034200094EC0EF00401460E826F94EC0EF0CAEF9D
:103430001EF0078432EC38F013EC31F02DC500F1AA
:103440009CEC30F004014C0E826F94EC0EF0040101
:10345000300E826F94EC0EF004012C0E826F94EC0F
:103460000EF031C182F40401300E822794EC0EF08C
:1034700032C182F40401300E822794EC0EF033C185
:1034800082F40401300E822794EC0EF004012C0E1D
:10349000826F94EC0EF013EC31F02EC500F19CEC31
:1034A00030F031C182F40401300E822794EC0EF02A
:1034B00032C182F40401300E822794EC0EF033C145
:1034C00082F40401300E822794EC0EF00794CAEFC8
:1034D0001EF004014C0E826F94EC0EF00401650E98
:1034E000826F94EC0EF0D2EC33F0CAEF1EF00401C0
:1034F0004C0E826F94EC0EF00401450E826F94EC3A
:103500000EF0E9EC33F0CAEF1EF004014C0E826FAE
:1035100094EC0EF00401620E826F94EC0EF017EC46
:1035200034F0CAEF1EF004014C0E826F94EC0EF0E2
:103530000401420E826F94EC0EF000EC34F0CAEFFE
:103540001EF004014C0E826F94EC0EF00401760E16
:10355000826F94EC0EF004012C0E826F94EC0EF04E
:1035600010A807D00401310E826F94EC0EF0CAEF60
:103570001EF00401300E826F94EC0EF0CAEF1EF0C4
:1035800004014C0E826F94EC0EF004015A0E826F0F
:1035900094EC0EF004012C0E826F94EC0EF032ECE1
:1035A00038F013EC31F005012E51130A06E0050145
:1035B0002E51170A0DE0F1EF1AF00101000E006F15
:1035C000000E016F100E026F000E036FF1EF1AF084
:1035D0000101000E006F000E016F000E026F010E60
:1035E000036F0101200E046F000E056F000E066FC1
:1035F000000E076F2FEC30F09CEC30F02AC182F403
:103600000401300E822794EC0EF02BC182F40401E9
:10361000300E822794EC0EF02CC182F40401300E9F
:10362000822794EC0EF02DC182F40401300E822723
:1036300094EC0EF02EC182F40401300E822794EC3B
:103640000EF02FC182F40401300E822794EC0EF0AC
:1036500030C182F40401300E822794EC0EF031C1A7
:1036600082F40401300E822794EC0EF032C182F411
:103670000401300E822794EC0EF033C182F4040171
:10368000300E822794EC0EF0CAEF1EF0078404017E
:103690004C0E826F94EC0EF00401310E826F94ECAC
:1036A0000EF004012C0E826F94EC0EF025C500F193
:1036B00026C501F127C502F128C503F10101200E3D
:1036C000046F000E056F000E066F000E076F2FECE3
:1036D00030F09CEC30F02AC182F40401300E8227D5
:1036E00094EC0EF02BC182F40401300E822794EC8E
:1036F0000EF02CC182F40401300E822794EC0EF0FF
:103700002DC182F40401300E822794EC0EF02EC1FC
:1037100082F40401300E822794EC0EF02FC182F463
:103720000401300E822794EC0EF030C182F40401C3
:10373000300E822794EC0EF031C182F40401300E79
:10374000822794EC0EF032C182F40401300E8227FD
:1037500094EC0EF033C182F40401300E822794EC15
:103760000EF00794CAEF1EF0078404014C0E826F1E
:1037700094EC0EF00401320E826F94EC0EF006EC25
:1037800036F00794CAEF1EF0078437B0CAEF1BF07B
:10379000DDEF1BF0010E166E04014C0E826F94ECEF
:1037A0000EF00401330E826F94EC0EF063EC36F0F1
:1037B000000E166E079451EF1BF0020E166E63ECAE
:1037C00036F08B800501010E306F3C0E316F010128
:1037D0005E6B5F6B606B616B626B636B646B656B85
:1037E000666B676B686B696B536B546BCF6ACE6AA1
:1037F0000F9A0F9C0F9E030E166E04014C0E826FE3
:1038000094EC0EF00401330E826F94EC0EF0040180
:103810002C0E826F94EC0EF004012D0E826F94EC4E
:103820000EF00401310E826F94EC0EF014EF2AF0CA
:1038300063EC36F0000E166E8B9016EF2AF00784BC
:1038400004014C0E826F94EC0EF00401340E826F72
:1038500094EC0EF004012C0E826F94EC0EF054ECFC
:1038600031F084C32AF185C32BF186C32CF187C3C1
:103870002DF188C32EF189C32FF18AC330F18BC398
:1038800031F18CC332F18DC333F10101296B61EC4D
:1038900031F0D8EC30F0200E046F000E056F000EF2
:1038A000066F000E076F0FEC30F000C121F501C16B
:1038B00022F502C123F503C124F5E5EC37F038C544
:1038C000AFF539C5B0F53AC5B1F53BC5B2F53CC564
:1038D000B3F53DC5B4F53EC5B5F5B9EC16F0040138
:1038E0002C0E826F94EC0EF03FC500F140C501F143
:1038F00041C502F142C503F10101000E046F000E43
:10390000056F010E066F000E076F2FEC30F09CEC78
:1039100030F029678EEF1CF093EF1CF004012D0EA0
:10392000826F94EC0EF030C182F40401300E8227D5
:1039300094EC0EF031C182F40401300E822794EC35
:103940000EF004012E0E826F94EC0EF032C182F460
:103950000401300E822794EC0EF033C182F404018E
:10396000300E822794EC0EF004012C0E826F94EC42
:103970000EF013EC31F043C500F144C501F140EC09
:103980002BF004012C0E826F94EC0EF013EC31F04E
:1039900045C500F19CEC30F031C182F40401300ED9
:1039A000822794EC0EF032C182F40401300E82279B
:1039B00094EC0EF033C182F40401300E822794ECB3
:1039C0000EF004012C0E826F94EC0EF037C5E8FF68
:1039D000E8B806D00401300E826F94EC0EF005D0EA
:1039E0000401310E826F94EC0EF004012C0E826FF4
:1039F00094EC0EF037C5E8FFE8BA06D00401300EAB
:103A0000826F94EC0EF06CD00401310E826F94EC56
:103A10000EF004012C0E826F94EC0EF047C500F1FD
:103A200048C501F149C502F14AC503F1BEEC30F0C9
:103A30005FEC2EF004012C0E826F94EC0EF04BC55F
:103A400000F14CC501F14DC502F14EC503F1010174
:103A5000000E046F000E056F010E066F000E076F5B
:103A60002FEC30F09CEC30F0296739EF1DF03EEF81
:103A70001DF004012D0E826F94EC0EF030C182F423
:103A80000401300E822794EC0EF031C182F404015F
:103A9000300E822794EC0EF004012E0E826F94EC0F
:103AA0000EF032C182F40401300E822794EC0EF045
:103AB00033C182F40401300E822794EC0EF004012D
:103AC0002C0E826F94EC0EF04FC500F150C501F141
:103AD00051C502F152C503F1BEEC30F05FEC2EF09F
:103AE0000794CAEF1EF054EC31F085C32AF186C367
:103AF0002BF187C32CF188C32DF189C32EF18AC322
:103B00002FF18BC330F18CC331F18DC332F18EC3F1
:103B100033F10101296B61EC31F0D8EC30F0010197
:103B2000010E046F000E056F000E066F000E076F8A
:103B3000FEEC2FF0100E046F000E056F000E066FE6
:103B4000000E076F0FEC30F000C129F501C12AF516
:103B500002C12BF503C12CF58DEC35F004014C0EA0
:103B6000826F94EC0EF00401460E826F94EC0EF01E
:103B700004012C0E826F94EC0EF025C500F126C5D1
:103B800001F127C502F128C503F10101100E046FF0
:103B9000000E056F000E066F000E076F2FEC30F061
:103BA0009CEC30F02AC182F40401300E822794ECA0
:103BB0000EF02BC182F40401300E822794EC0EF03B
:103BC0002CC182F40401300E822794EC0EF02DC13A
:103BD00082F40401300E822794EC0EF02EC182F4A0
:103BE0000401300E822794EC0EF02FC182F4040100
:103BF000300E822794EC0EF030C182F40401300EB6
:103C0000822794EC0EF031C182F40401300E822739
:103C100094EC0EF032C182F40401300E822794EC51
:103C20000EF033C182F40401300E822794EC0EF0C2
:103C3000CAEF1EF037B01FEF1EF0020E166E63ECD7
:103C400036F000011650020AD8B43DEF1EF005010F
:103C50002F51010AD8B433EF1EF015B238EF1EF021
:103C600081BA38EF1EF0000E166E158416EF2AF09A
:103C7000050E166E1584D8EF38F08B8001015E6B4F
:103C80005F6B606B616B626B636B646B656B666BC8
:103C9000676B686B696B536B546BCF6ACE6A0F9A14
:103CA0000F9C0F9E030E166E16EF2AF063EC36F093
:103CB00005012F51010AD8B464EF1EF015B269EF67
:103CC0001EF081BA69EF1EF0000E166E158416EF15
:103CD0002AF0050E166E1584D8EF38F004014C0E4C
:103CE000826F94EC0EF00401350E826F94EC0EF0AE
:103CF00004012C0E826F94EC0EF013EC31F007846B
:103D0000B9C500F107949CEC30F031C182F4040194
:103D1000300E822794EC0EF032C182F40401300E92
:103D2000822794EC0EF033C182F40401300E822716
:103D300094EC0EF0CAEF1EF026EC36F013EC31F0E6
:103D400037C500F19CEC30F004014C0E826F94EC0E
:103D50000EF00401360E826F94EC0EF004012C0E6E
:103D6000826F94EC0EF031C182F40401300E822790
:103D700094EC0EF032C182F40401300E822794ECF0
:103D80000EF033C182F40401300E822794EC0EF061
:103D9000CAEF1EF09EEC0EF016EF2AF004014C0E56
:103DA000826F94EC0EF00401500E826F94EC0EF0D2
:103DB00004012C0E826F94EC0EF085C32AF186C3A9
:103DC0002BF187C32CF188C32DF189C32EF18AC34F
:103DD0002FF18BC330F18CC331F18DC332F18EC31F
:103DE00033F1010161EC31F0D8EC30F00301845182
:103DF000530A0DE0030184514D0A38E00401780EA6
:103E0000826F94EC0EF09EEC0EF016EF2AF0040197
:103E1000530E826F94EC0EF0250E0C6E00C10BF069
:103E20004DEC0BF0260E0C6E01C10BF04DEC0BF0BF
:103E3000270E0C6E02C10BF04DEC0BF0280E0C6E31
:103E400003C10BF04DEC0BF000C157F501C158F563
:103E500002C159F503C15AF500C15BF501C15CF51A
:103E600002C15DF503C15EF5ABEF1FF004014D0E1D
:103E7000826F94EC0EF0290E0C6E00C10BF04DEC2D
:103E80000BF000C15FF500C160F5ABEF1FF004015E
:103E90004C0E826F94EC0EF00401540E826F94EC81
:103EA0000EF004012C0E826F94EC0EF084C32AF104
:103EB00085C32BF186C32CF187C32DF188C32EF166
:103EC00089C32FF18AC330F18BC331F18DC332F135
:103ED0008EC333F1010161EC31F0D8EC30F0010117
:103EE000000E046F000E056F010E066F000E076FC7
:103EF0000FEC30F0210E0C6E00C10BF04DEC0BF00E
:103F0000220E0C6E01C10BF04DEC0BF0230E0C6E6B
:103F100002C10BF04DEC0BF0240E0C6E03C10BF044
:103F20004DEC0BF000C161F501C162F502C163F512
:103F300003C164F5ABEF1FF004014C0E826F94ECEB
:103F40000EF00401490E826F94EC0EF004012C0E69
:103F5000826F94EC0EF0250E64EC0BF0E8CF00F1CC
:103F6000260E64EC0BF0E8CF01F1270E64EC0BF0A9
:103F7000E8CF02F1280E64EC0BF0E8CF03F19CECE3
:103F800030F05FEC2EF00401730E826F94EC0EF0B3
:103F900004012C0E826F94EC0EF013EC31F0290E1C
:103FA00064EC0BF0E8CF00F19CEC30F05FEC2EF00D
:103FB00004016D0E826F94EC0EF004012C0E826FE2
:103FC00094EC0EF05BC500F15CC501F15DC502F13A
:103FD0005EC503F19CEC30F05FEC2EF00401730E33
:103FE000826F94EC0EF004012C0E826F94EC0EF0B4
:103FF00013EC31F060C500F19CEC30F05FEC2EF07A
:1040000004016D0E826F94EC0EF004012C0E826F91
:1040100094EC0EF061C500F162C501F163C502F1D7
:1040200064C503F131EC2AF004012C0E826F94EC8C
:104030000EF09EEC0EF016EF2AF083C32AF184C333
:104040002BF185C32CF186C32DF187C32EF188C3D4
:104050002FF189C330F18AC331F18BC332F18CC3A4
:1040600033F1010161EC31F0D8EC30F0160E0C6E3A
:1040700000C10BF04DEC0BF0170E0C6E01C10BF0F4
:104080004DEC0BF0180E0C6E02C10BF04DEC0BF06A
:10409000190E0C6E03C10BF04DEC0BF000C18EF14C
:1040A00001C18FF102C190F103C191F100C192F100
:1040B00001C193F102C194F103C195F1FFEF20F02A
:1040C00083C32AF184C32BF185C32CF186C32DF160
:1040D00087C32EF188C32FF189C330F18AC331F130
:1040E0008BC332F18CC333F1010161EC31F0D8ECB8
:1040F00030F000C18EF101C18FF102C190F103C116
:1041000091F100C192F101C193F102C194F103C197
:1041100095F1FFEF20F083C32AF184C32BF185C30F
:104120002CF186C32DF187C32EF188C32FF189C3EB
:1041300030F18AC331F18CC332F18DC333F1010107
:1041400061EC31F0D8EC30F00101000E046F000E8C
:10415000056F010E066F000E076F0FEC30F01A0EA0
:104160000C6E00C10BF04DEC0BF01B0E0C6E01C180
:104170000BF04DEC0BF01C0E0C6E02C10BF04DEC75
:104180000BF01D0E0C6E03C10BF04DEC0BF000C1DB
:1041900096F101C197F102C198F103C199F1FFEFC6
:1041A00020F083C32AF184C32BF185C32CF186C38D
:1041B0002DF187C32EF188C32FF189C330F18AC353
:1041C00031F18CC332F18DC333F1010161EC31F077
:1041D000D8EC30F00101000E046F000E056F010EE7
:1041E000066F000E076F0FEC30F000C196F101C1B1
:1041F00097F102C198F103C199F1FFEF20F0160E7B
:1042000064EC0BF0E8CF00F1170E64EC0BF0E8CF94
:1042100001F1180E64EC0BF0E8CF02F1190E64EC1A
:104220000BF0E8CF03F19CEC30F05FEC2EF00401D2
:10423000730E826F94EC0EF004012C0E826F94ECDE
:104240000EF08EC100F18FC101F190C102F191C158
:1042500003F19CEC30F05FEC2EF00401730E826FE2
:1042600094EC0EF004012C0E826F94EC0EF01A0EFA
:1042700064EC0BF0E8CF00F11B0E64EC0BF0E8CF20
:1042800001F11C0E64EC0BF0E8CF02F11D0E64ECA2
:104290000BF0E8CF03F131EC2AF004012C0E826F11
:1042A00094EC0EF096C100F197C101F198C102F1B2
:1042B00099C103F131EC2AF09EEC0EF016EF2AF0D2
:1042C0000401690E826F94EC0EF004012C0E826FD3
:1042D00094EC0EF00101040E006F000E016F000E51
:1042E000026F000E036F9CEC30F02CC182F40401CD
:1042F000300E822794EC0EF02DC182F40401300EB2
:10430000822794EC0EF02EC182F40401300E822735
:1043100094EC0EF02FC182F40401300E822794EC4D
:104320000EF030C182F40401300E822794EC0EF0BE
:1043300031C182F40401300E822794EC0EF032C1B8
:1043400082F40401300E822794EC0EF033C182F423
:104350000401300E822794EC0EF004012C0E826FC3
:1043600094EC0EF001010D0E006F000E016F000EB7
:10437000026F000E036F9CEC30F02CC182F404013C
:10438000300E822794EC0EF02DC182F40401300E21
:10439000822794EC0EF02EC182F40401300E8227A5
:1043A00094EC0EF02FC182F40401300E822794ECBD
:1043B0000EF030C182F40401300E822794EC0EF02E
:1043C00031C182F40401300E822794EC0EF032C128
:1043D00082F40401300E822794EC0EF033C182F493
:1043E0000401300E822794EC0EF004012C0E826F33
:1043F00094EC0EF00101480E006F000E016F000EEC
:10440000026F000E036F9CEC30F02CC182F40401AB
:10441000300E822794EC0EF02DC182F40401300E90
:10442000822794EC0EF02EC182F40401300E822714
:1044300094EC0EF02FC182F40401300E822794EC2C
:104440000EF030C182F40401300E822794EC0EF09D
:1044500031C182F40401300E822794EC0EF032C197
:1044600082F40401300E822794EC0EF033C182F402
:104470000401300E822794EC0EF004012C0E826FA2
:1044800094EC0EF0200EF86EF76AF66A040109004B
:10449000F5CF82F494EC0EF00900F5CF82F494ECA1
:1044A0000EF00900F5CF82F494EC0EF00900F5CF80
:1044B00082F494EC0EF00900F5CF82F494EC0EF047
:1044C0000900F5CF82F494EC0EF00900F5CF82F4E8
:1044D00094EC0EF00900F5CF82F494EC0EF09EEC13
:1044E0000EF016EF2AF08351630AD8A414EF2AF0D5
:1044F0008451610AD8A414EF2AF085516C0AD8A41B
:1045000014EF2AF08651410A3FE08651440A1BE02D
:104510008651420AD8B4D7EF22F08651350AD8B472
:10452000A0EF2BF08651360AD8B4F5EF2BF0865168
:10453000370AD8B45EEF2CF08651380AD8B4BCEFF5
:104540002CF014EF2AF00798079A04017A0E826F74
:1045500094EC0EF00401780E826F94EC0EF00401DE
:10456000640E826F94EC0EF00401550E826F94EC91
:104570000EF0C0EF22F004014C0E826F94EC0EF0AE
:104580009EEC0EF016EF2AF00788079A04017A0EC7
:10459000826F94EC0EF00401410E826F94EC0EF0E9
:1045A0000401610E826F94EC0EF0B4EF22F00798D4
:1045B000078A04017A0E826F94EC0EF00401420E19
:1045C000826F94EC0EF00401610E826F94EC0EF099
:1045D000B4EF22F001016667F5EF22F06767F5EFAF
:1045E00022F06867F5EF22F0696716D001014F6786
:1045F00001EF23F0506701EF23F0516701EF23F043
:1046000052670AD00101000E006F000E016F000E0C
:10461000026F000E036F120011B80AD00101620E82
:10462000046F010E056F000E066F000E076F09D0B4
:104630000101A70E046F020E056F000E066F000E3B
:10464000076F66C100F167C101F168C102F169C17C
:1046500003F1FEEC2FF003BF9EEF23F0119A119CA3
:104660000101000E046FA80E056F550E066F020EB5
:10467000076F66C100F167C101F168C102F169C14C
:1046800003F166C18AF167C18BF168C18CF169C120
:104690008DF1FEEC2FF003BF0BD00101000E8A6FED
:1046A000A80E8B6F550E8C6F020E8D6F118A119CA8
:1046B0000E0E64EC0BF0E8CF18F10F0E64EC0BF06B
:1046C000E8CF19F1100E64EC0BF0E8CF1AF1110EDF
:1046D00064EC0BF0E8CF1BF147EC2FF08AC104F13A
:1046E0008BC105F18CC106F18DC107F1FEEC2FF0F5
:1046F00007820BEC2FF047EC2FF007920BEC2FF01A
:104700008AC100F18BC101F18CC102F18DC103F1AD
:1047100007920BEC2FF0CC0E046FE00E056F870EA6
:10472000066F050E076FFEEC2FF000C118F101C1F6
:1047300019F102C11AF103C11BF140D013AAA3EF72
:1047400023F0138E139A119C119A0101800E006FB1
:104750001A0E016F060E026F000E036F4FC104F1B7
:1047600050C105F151C106F152C107F1FEEC2FF025
:1047700003AF05D013EC31F0118C119A12000E0E1C
:1047800064EC0BF0E8CF18F10F0E64EC0BF0E8CFFF
:1047900019F1100E64EC0BF0E8CF1AF1110E64EC75
:1047A0000BF0E8CF1BF14FC100F150C101F151C135
:1047B00002F152C103F107820BEC2FF018C100F196
:1047C00019C101F11AC102F11BC103F112000784E2
:1047D000BAC166F1BBC167F1BCC168F1BDC169F185
:1047E0004BC14FF14CC150F14DC151F14EC152F18D
:1047F00057C159F158C15AF107940101666708EF92
:1048000024F0676708EF24F0686708EF24F0696711
:1048100016D001014F6714EF24F0506714EF24F015
:10482000516714EF24F052670AD00101000E006FA7
:10483000000E016F000E026F000E036F120011B820
:104840000AD00101620E046F010E056F000E066FA3
:10485000000E076F09D00101A70E046F020E056F4D
:10486000000E066F000E076F66C100F167C101F10F
:1048700068C102F169C103F1FEEC2FF003BFA0EFA4
:1048800024F00101000E046FA80E056F550E066F8F
:10489000020E076F66C100F167C101F168C102F144
:1048A00069C103F166C18AF167C18BF168C18CF1FE
:1048B00069C18DF1FEEC2FF003BF09D00101000E9C
:1048C0008A6FA80E8B6F550E8C6F020E8D6F47ECA2
:1048D0002FF000C104F101C105F102C106F103C1CD
:1048E00007F1000E006FA00E016F980E026F7B0E95
:1048F000036F2FEC30F000C118F101C119F102C1B2
:104900001AF103C11BF1000E006FA00E016F980E8B
:10491000026F7B0E036F8AC104F18BC105F18CC15C
:1049200006F18DC107F12FEC30F018C104F119C167
:1049300005F11AC106F11BC107F1FEEC2FF01200C0
:104940000101A80E006F610E016F000E026F000ED4
:10495000036F4FC104F150C105F151C106F152C1BD
:1049600007F1FEEC2FF003AF0AD00101A80E006F93
:10497000610E016F000E026F000E036F00D0C80EB3
:10498000006FAF0E016F000E026F000E036F4FC17C
:1049900004F150C105F151C106F152C107F10FEC0C
:1049A00030F012000401730E826F94EC0EF00401DB
:1049B0002C0E826F94EC0EF0078462C166F163C125
:1049C00067F164C168F165C169F14BC14FF14CC138
:1049D00050F14DC151F14EC152F157C159F158C179
:1049E0005AF10794F8EC24F09EEC0EF016EF2AF042
:1049F00066C100F167C101F168C102F169C103F14B
:104A000001019CEC30F05FEC2EF00401630E826F2C
:104A100094EC0EF004012C0E826F94EC0EF04FC15A
:104A200000F150C101F151C102F152C103F1010184
:104A30009CEC30F05FEC2EF00401660E826F94EC7B
:104A40000EF004012C0E826F94EC0EF013EC31F09A
:104A500059C100F15AC101F101019CEC30F05FEC49
:104A60002EF00401740E826F94EC0EF0120010828E
:104A70000401530E826F94EC0EF004012C0E826F31
:104A800094EC0EF083C32AF184C32BF185C32CF17F
:104A900086C32DF187C32EF188C32FF189C330F16E
:104AA0008AC331F18BC332F18CC333F1010161EC64
:104AB00031F0D8EC30F000C166F101C167F102C1FC
:104AC00068F103C169F18EC32AF18FC32BF190C342
:104AD0002CF191C32DF192C32EF193C32FF194C306
:104AE00030F195C331F196C332F197C333F101012F
:104AF00061EC31F0D8EC30F000C14FF101C150F160
:104B000002C151F103C152F154EC31F099C32FF1BC
:104B10009AC330F19BC331F19CC332F19DC333F191
:104B2000010161EC31F0D8EC30F000C159F101C164
:104B30005AF1F8EC24F004012C0E826F94EC0EF084
:104B4000B2EF25F0118E1CA002D01CAE108C1BBE43
:104B500002D01BA4108E03018251520A02E10F827F
:104B600001D00F928251750A02E1108401D0109495
:104B70008251550A02E1108601D010968351310A04
:104B800003E11382138402D013921394030183511F
:104B9000660A01E056D00401660E826F94EC0EF0B6
:104BA00004012C0E826F94EC0EF0E7EC23F09CECE9
:104BB00030F02AC182F40401300E822794EC0EF00A
:104BC0002BC182F40401300E822794EC0EF02CC12C
:104BD00082F40401300E822794EC0EF02DC182F491
:104BE0000401300E822794EC0EF02EC182F40401F1
:104BF000300E822794EC0EF02FC182F40401300EA7
:104C0000822794EC0EF030C182F40401300E82272A
:104C100094EC0EF031C182F40401300E822794EC42
:104C20000EF032C182F40401300E822794EC0EF0B3
:104C300033C182F40401300E822794EC0EF014EF9D
:104C40002AF011A003D011A401D01084078410B25F
:104C50008BEF26F010A46FEF26F0BAC166F1BBC14E
:104C600067F1BCC168F1BDC169F1BEC16AF1BFC1E4
:104C70006BF1C0C16CF1C1C16DF1C2C16EF1C3C1B4
:104C80006FF1C4C170F1C5C171F1C6C172F1C7C184
:104C900073F1C8C174F1C9C175F1CAC176F1CBC154
:104CA00077F1CCC178F1CDC179F1CEC17AF1CFC124
:104CB0007BF1D0C17CF1D1C17DF1D2C17EF1D3C1F4
:104CC0007FF1D4C180F1D5C181F1D6C182F1D7C1C4
:104CD00083F1D8C184F1D9C185F177EF26F062C1A3
:104CE00066F163C167F164C168F165C169F1BAC178
:104CF00086F1BBC187F1BCC188F1BDC189F14BC14F
:104D00004FF14CC150F14DC151F14EC152F157C15B
:104D100059F158C15AF107940FA0ADEF26F00101E7
:104D200096679AEF26F097679AEF26F098679AEFC2
:104D300026F099679EEF26F0ADEF26F0EAEC22F020
:104D400096C104F197C105F198C106F199C107F127
:104D5000FEEC2FF003BFDAEF29F0EAEC22F00101BC
:104D6000000E046F000E056F010E066F000E076F38
:104D70002FEC30F011A02AD011A228D09CEC30F0FA
:104D8000296701D005D004012D0E826F94EC0EF03E
:104D900030C182F40401300E822794EC0EF031C150
:104DA00082F40401300E822794EC0EF032C182F4BA
:104DB0000401300E822794EC0EF033C182F404011A
:104DC000300E822794EC0EF09EEC0EF012A8C5D0A7
:104DD00012981DC01EF01E3A1E42070E1E1600013C
:104DE0001E50000AD8B479EF27F000011E50010AC6
:104DF000D8B405EF27F000011E50020AD8B403EF23
:104E000027F0ABEF27F0ABEF27F013EC31F02DC01C
:104E100001F12EC000F1D89001330033D890013356
:104E200000330101630E046F000E056F000E066F64
:104E3000000E076F2FEC30F0280E046F000E056F88
:104E4000000E066F000E076FFEEC2FF000C130F071
:104E500013EC31F02BC001F1019F019D2CC000F13A
:104E60000101A40E046F000E056F000E066F000E08
:104E7000076F2FEC30F000C12FF000C104F101C129
:104E800005F102C106F103C107F1640E006F000EC7
:104E9000016F000E026F000E036FFEEC2FF0050E87
:104EA000046F000E056F000E066F000E076F2FECEB
:104EB00030F000C104F101C105F102C106F103C1E6
:104EC00007F113EC31F030C000F1FEEC2FF000C11F
:104ED00031F031C0E8FF050F305C03E78A84ABEFA7
:104EE00027F031C0E8FF0A0F305C01E68A94ABEF8F
:104EF00027F000C124F101C125F102C126F103C14F
:104F000027F113EC31F019EC31F01D501F0BE8CFF5
:104F100000F10101640E046F000E056F000E066FB4
:104F2000000E076F0FEC30F024C104F125C105F12C
:104F300026C106F127C107F1FEEC2FF003BF02D016
:104F40008A9401D08A8424C100F125C101F126C1CF
:104F500002F127C103F116EF2AF000C124F101C1CB
:104F600025F102C126F103C127F110AE4DD0109EEC
:104F700000C108F101C109F102C10AF103C10BF13D
:104F80009CEC30F030C1E2F131C1E3F132C1E4F127
:104F900033C1E5F108C100F109C101F10AC102F113
:104FA0000BC103F101016C0E046F070E056F000EBB
:104FB000066F000E076FFEEC2FF003BF04D0010157
:104FC000550EE66F1CD008C100F109C101F10AC1FC
:104FD00002F10BC103F10101A40E046F060E056F6F
:104FE000000E066F000E076FFEEC2FF003BF04D01B
:104FF00001017F0EE66F03D00101FF0EE66F1F8EE9
:1050000011AEDAEF29F0119E24C100F125C101F1A2
:1050100026C102F127C103F111A005D011A203D0CE
:105020000FB0DAEF29F010A41DEF28F00401750E7F
:10503000826F94EC0EF022EF28F00401720E826F62
:1050400094EC0EF004012C0E826F94EC0EF09CECAC
:1050500030F0296731EF28F00401200E826F34EF21
:1050600028F004012D0E826F94EC0EF030C182F412
:105070000401300E822794EC0EF031C182F4040159
:10508000300E822794EC0EF004012E0E826F94EC09
:105090000EF032C182F40401300E822794EC0EF03F
:1050A00033C182F40401300E822794EC0EF0040127
:1050B0006D0E826F94EC0EF004012C0E826F94EC56
:1050C0000EF04FC100F150C101F151C102F152C1C6
:1050D00003F101019CEC30F05FEC2EF00401480E6E
:1050E000826F94EC0EF004017A0E826F94EC0EF055
:1050F00004012C0E826F94EC0EF066C100F167C1C2
:1051000001F168C102F169C103F101019CEC30F0C9
:105110005FEC2EF00401630E826F94EC0EF004013C
:105120002C0E826F94EC0EF066C100F167C101F1A4
:1051300068C102F169C103F101010A0E046F000E9A
:10514000056F000E066F000E076F0FEC30F0000EBB
:10515000046F120E056F000E066F000E076F2FEC26
:1051600030F09CEC30F02AC182F40401300E82272A
:1051700094EC0EF02BC182F40401300E822794ECE3
:105180000EF02CC182F40401300E822794EC0EF054
:105190002DC182F40401300E822794EC0EF02EC152
:1051A00082F40401300E822794EC0EF02FC182F4B9
:1051B0000401300E822794EC0EF030C182F4040119
:1051C000300E822794EC0EF004012E0E826F94ECC8
:1051D0000EF031C182F40401300E822794EC0EF0FF
:1051E00032C182F40401300E822794EC0EF033C1F8
:1051F00082F40401300E822794EC0EF00401730E49
:10520000826F94EC0EF004012C0E826F94EC0EF081
:1052100013EC31F059C100F15AC101F140EC2BF00F
:1052200013A262EF29F004012C0E826F94EC0EF0B1
:1052300086C166F187C167F188C168F189C169F1EA
:10524000EAEC22F00101000E046F000E056F010E62
:10525000066F000E076F2FEC30F09CEC30F02967E2
:1052600037EF29F00401200E826F3AEF29F0040194
:105270002D0E826F94EC0EF030C182F40401300EDA
:10528000822794EC0EF031C182F40401300E8227A3
:1052900094EC0EF004012E0E826F94EC0EF032C1ED
:1052A00082F40401300E822794EC0EF033C182F4B4
:1052B0000401300E822794EC0EF004016D0E826F13
:1052C00094EC0EF013A489EF29F004012C0E826FE8
:1052D00094EC0EF013AC77EF29F00401500E826FBE
:1052E00094EC0EF0139C1398139A89EF29F013AEE7
:1052F00084EF29F00401460E826F94EC0EF0139EA9
:105300001398139A89EF29F00401530E826F94ECDD
:105310000EF037B0A0EF29F004012C0E826F94EC50
:105320000EF08BB09BEF29F00401440E826F94ECD9
:105330000EF0A0EF29F00401530E826F94EC0EF0F2
:105340000FB2A6EF29F00FA0D8EF29F004012C0E20
:10535000826F94EC0EF0200EF86EF76AF66A040184
:105360000900F5CF82F494EC0EF00900F5CF82F439
:1053700094EC0EF00900F5CF82F494EC0EF00900E5
:10538000F5CF82F494EC0EF00900F5CF82F494ECA2
:105390000EF00900F5CF82F494EC0EF00900F5CF81
:1053A00082F494EC0EF00900F5CF82F494EC0EF048
:1053B0009EEC0EF00F90109E129816EF2AF004014A
:1053C000630E826F94EC0EF004012C0E826F94EC4D
:1053D0000EF01CEC2AF004012C0E826F94EC0EF0FF
:1053E0008FEC2AF004012C0E826F94EC0EF00BEC83
:1053F0002BF004012C0E826F94EC0EF00101F80EDC
:10540000006FCD0E016F660E026F030E036F31EC5D
:105410002AF004012C0E826F94EC0EF021EC2BF09C
:105420009EEC0EF016EF2AF09EEC0EF00301C26B1C
:105430000790109225EF2DF0D8900E0E64EC0BF033
:10544000E8CF00F10F0E64EC0BF0E8CF01F1100E85
:1054500064EC0BF0E8CF02F1110E64EC0BF0E8CF36
:1054600003F10101000E046F000E056F010E066FBF
:10547000000E076F2FEC30F09CEC30F02AC182F464
:105480000401300E822794EC0EF02BC182F404014B
:10549000300E822794EC0EF02CC182F40401300E01
:1054A000822794EC0EF02DC182F40401300E822785
:1054B00094EC0EF02EC182F40401300E822794EC9D
:1054C0000EF02FC182F40401300E822794EC0EF00E
:1054D00030C182F40401300E822794EC0EF031C109
:1054E00082F40401300E822794EC0EF004012E0E9B
:1054F000826F94EC0EF032C182F40401300E8227E8
:1055000094EC0EF033C182F40401300E822794EC47
:105510000EF004016D0E826F94EC0EF01200120E6C
:1055200064EC0BF0E8CF00F1130E64EC0BF0E8CF65
:1055300001F1140E64EC0BF0E8CF02F1150E64ECEF
:105540000BF0E8CF03F101010A0E046F000E056FA6
:10555000000E066F000E076F0FEC30F0000E046FA8
:10556000120E056F000E066F000E076F2FEC30F065
:105570009CEC30F02AC182F40401300E822794ECB6
:105580000EF02BC182F40401300E822794EC0EF051
:105590002CC182F40401300E822794EC0EF02DC150
:1055A00082F40401300E822794EC0EF02EC182F4B6
:1055B0000401300E822794EC0EF02FC182F4040116
:1055C000300E822794EC0EF030C182F40401300ECC
:1055D000822794EC0EF004012E0E826F94EC0EF0F4
:1055E00031C182F40401300E822794EC0EF032C1F6
:1055F00082F40401300E822794EC0EF033C182F461
:105600000401300E822794EC0EF00401730E826FB9
:1056100094EC0EF012000A0E64EC0BF0E8CF00F1EF
:105620000B0E64EC0BF0E8CF01F10C0E64EC0BF008
:10563000E8CF02F10D0E64EC0BF0E8CF03F140EF80
:105640002BF0060E64EC0BF0E8CF00F1070E64ECD3
:105650000BF0E8CF01F1080E64EC0BF0E8CF02F19B
:10566000090E64EC0BF0E8CF03F140EF2BF00101E1
:1056700013EC31F0078457C100F158C101F10794D0
:105680000101E80E046F800E056F000E066F000E1C
:10569000076F0FEC30F0000E046F040E056F000E64
:1056A000066F000E076F2FEC30F0880E046F130E9C
:1056B000056F000E066F000E076FFEEC2FF00A0E4E
:1056C000046F000E056F000E066F000E076F2FECC3
:1056D00030F09CEC30F00101296774EF2BF00401ED
:1056E000200E826F77EF2BF004012D0E826F94EC69
:1056F0000EF030C182F40401300E822794EC0EF0DB
:1057000031C182F40401300E822794EC0EF032C1D4
:1057100082F40401300E822794EC0EF004012E0E68
:10572000826F94EC0EF033C182F40401300E8227B4
:1057300094EC0EF00401430E826F94EC0EF0120014
:1057400087C32AF188C32BF189C32CF18AC32DF1B9
:105750008BC32EF18CC32FF18DC330F18EC331F189
:1057600090C332F191C333F10101296B61EC31F047
:10577000D8EC30F00101000E046F000E056F010E31
:10578000066F000E076F0FEC30F00E0E0C6E00C1AE
:105790000BF04DEC0BF00F0E0C6E01C10BF04DEC4D
:1057A0000BF0100E0C6E02C10BF04DEC0BF0110E55
:1057B0000C6E03C10BF04DEC0BF004017A0E826FFE
:1057C00094EC0EF004012C0E826F94EC0EF00401A8
:1057D000350E826F94EC0EF004012C0E826F94EC67
:1057E0000EF01CEC2AF0C0EF22F087C32AF188C328
:1057F0002BF189C32CF18AC32DF18BC32EF18CC3FD
:105800002FF18DC330F18EC331F190C332F191C3CA
:1058100033F10101296B61EC31F0D8EC30F0880EE6
:10582000046F130E056F000E066F000E076F03EC7A
:1058300030F0000E046F040E056F000E066F000EB0
:10584000076F0FEC30F00101E80E046F800E056F5A
:10585000000E066F000E076F2FEC30F00A0E0C6E74
:1058600000C10BF04DEC0BF00B0E0C6E01C10BF0F8
:105870004DEC0BF00C0E0C6E02C10BF04DEC0BF06E
:105880000D0E0C6E03C10BF04DEC0BF004017A0E03
:10589000826F94EC0EF004012C0E826F94EC0EF0EB
:1058A0000401360E826F94EC0EF004012C0E826F10
:1058B00094EC0EF00BEC2BF0C0EF22F087C32AF132
:1058C00088C32BF189C32CF18AC32DF18BC32EF130
:1058D0008CC32FF18DC330F18FC331F190C332F1FE
:1058E00091C333F1010161EC31F0D8EC30F0000EDE
:1058F000046F120E056F000E066F000E076F0FEC9F
:1059000030F001010A0E046F000E056F000E066FE5
:10591000000E076F2FEC30F0120E0C6E00C10BF072
:105920004DEC0BF0130E0C6E01C10BF04DEC0BF0B7
:10593000140E0C6E02C10BF04DEC0BF0150E0C6E3C
:1059400003C10BF04DEC0BF004017A0E826F94EC66
:105950000EF004012C0E826F94EC0EF00401370E51
:10596000826F94EC0EF004012C0E826F94EC0EF01A
:105970008FEC2AF0C0EF22F087C32AF188C32BF105
:1059800089C32CF18AC32DF18BC32EF18CC32FF167
:105990008DC330F18EC331F190C332F191C333F135
:1059A0000101296B61EC31F0D8EC30F0880E046F06
:1059B000130E056F000E066F000E076F03EC30F03C
:1059C000000E046F040E056F000E066F000E076FC9
:1059D0000FEC30F00101E80E046F800E056F000E31
:1059E000066F000E076F2FEC30F0060E0C6E00C134
:1059F0000BF04DEC0BF0070E0C6E01C10BF04DECF3
:105A00000BF0080E0C6E02C10BF04DEC0BF0090E02
:105A10000C6E03C10BF04DEC0BF004017A0E826F9B
:105A200094EC0EF004012C0E826F94EC0EF0040145
:105A3000380E826F94EC0EF004012C0E826F94EC01
:105A40000EF021EC2BF0C0EF22F007A898EF2DF01C
:105A50000101800E006F1A0E016F060E026F000E1C
:105A6000036F4BC104F14CC105F14DC106F14EC1AC
:105A700007F1FEEC2FF003BFDEEF2DF059EC2EF016
:105A80004BC100F14CC101F14DC102F14EC103F116
:105A900007820BEC2FF018C104F119C105F11AC1EE
:105AA00006F11BC107F1F80E006FCD0E016F660EF7
:105AB000026F030E036FFEEC2FF00E0E0C6E00C192
:105AC0000BF04DEC0BF00F0E0C6E01C10BF04DEC1A
:105AD0000BF0100E0C6E02C10BF04DEC0BF0110E22
:105AE0000C6E03C10BF04DEC0BF00784010113ECBD
:105AF00031F057C100F158C101F107940A0E0C6E44
:105B000000C10BF04DEC0BF00B0E0C6E01C10BF055
:105B10004DEC0BF00C0E0C6E02C10BF04DEC0BF0CB
:105B20000D0E0C6E03C10BF04DEC0BF0DEEF2DF003
:105B300007AADEEF2DF00784010113EC31F057C105
:105B400000F158C101F10794060E0C6E00C10BF074
:105B50004DEC0BF0070E0C6E01C10BF04DEC0BF091
:105B6000080E0C6E02C10BF04DEC0BF0090E0C6E22
:105B700003C10BF04DEC0BF0078462C100F163C16F
:105B800001F164C102F165C103F10794120E0C6EBC
:105B900000C10BF04DEC0BF0130E0C6E01C10BF0BD
:105BA0004DEC0BF0140E0C6E02C10BF04DEC0BF033
:105BB000150E0C6E03C10BF04DEC0BF00798079A15
:105BC0000401805181197F0B0DE09EA8FED714EED1
:105BD00000F081517F0BE126E750812B0F01AD6E64
:105BE000E0EF2DF005012F51000AD8B421EF2EF07F
:105BF00081BA06EF2EF015B221EF2EF005012F51DC
:105C0000010AD8B41FEF2EF018EF2EF005012F5126
:105C1000000AD8B4D8EF38F005012F51010AD8B4E2
:105C20001FEF2EF000011650050AD8B4D8EF38F057
:105C300081B821EF2EF05CEC32F05AEC33F071ECCD
:105C400038F0C2EF0DF018C100F119C101F11AC10D
:105C500002F11BC103F1000E046F000E056F010E6F
:105C6000066F000E076F2FEC30F029A14EEF2EF0DB
:105C70002051D8B44EEF2EF018C100F119C101F136
:105C80001AC102F11BC103F1000E046F000E056F73
:105C90000A0E066F000E076F2FEC30F012000101A4
:105CA0000451001305510113065102130751031348
:105CB00012000101186B196B1A6B1B6B12002AC1C1
:105CC00082F40401300E822794EC0EF02BC182F492
:105CD0000401300E822794EC0EF02CC182F40401F2
:105CE000300E822794EC0EF02DC182F40401300EA8
:105CF000822794EC0EF02EC182F40401300E82272C
:105D000094EC0EF02FC182F40401300E822794EC43
:105D10000EF030C182F40401300E822794EC0EF0B4
:105D200031C182F40401300E822794EC0EF032C1AE
:105D300082F40401300E822794EC0EF033C182F419
:105D40000401300E822794EC0EF012002FC182F471
:105D50000401300E822794EC0EF030C182F404016D
:105D6000300E822794EC0EF031C182F40401300E23
:105D7000822794EC0EF032C182F40401300E8227A7
:105D800094EC0EF033C182F40401300E822794ECBF
:105D90000EF01200060E216E060E226E060E236E07
:105DA000212ED0EF2EF0222ED0EF2EF0232ED0EF8A
:105DB0002EF08B84020E216E020E226E020E236ED6
:105DC000212EE0EF2EF0222EE0EF2EF0232EE0EF3A
:105DD0002EF08B941200FF0E226E22C023F0030ED1
:105DE000216E8B84212EF1EF2EF0030E216E232ED7
:105DF000F1EF2EF08B9422C023F0030E216E212EA2
:105E0000FFEF2EF0030E216E233EFFEF2EF0222E29
:105E1000EDEF2EF012000101005305E1015303E103
:105E2000025301E1002BCEEC2FF013EC31F039518D
:105E3000006F3A51016F420E046F4B0E056F000E5A
:105E4000066F000E076F0FEC30F000C104F101C1C6
:105E500005F102C106F103C107F118C100F119C132
:105E600001F11AC102F11BC103F107B23CEF2FF09F
:105E700003EC30F03EEF2FF0FEEC2FF000C118F1F4
:105E800001C119F102C11AF103C11BF1120013EC97
:105E900031F059C100F15AC101F1060E64EC0BF06A
:105EA000E8CF04F1070E64EC0BF0E8CF05F1080E23
:105EB00064EC0BF0E8CF06F1090E64EC0BF0E8CFD0
:105EC00007F1FEEC2FF000C124F101C125F102C160
:105ED00026F103C127F1290E046F000E056F000E95
:105EE000066F000E076F0FEC30F0EE0E046F430EDE
:105EF000056F000E066F000E076F03EC30F024C133
:105F000004F125C105F126C106F127C107F10FEC07
:105F100030F000C11CF101C11DF102C11EF103C12D
:105F20001FF1120E64EC0BF0E8CF04F1130E64ECD9
:105F30000BF0E8CF05F1140E64EC0BF0E8CF06F19E
:105F4000150E64EC0BF0E8CF07F10D0E006F000E9C
:105F5000016F000E026F000E036F0FEC30F0180E91
:105F6000046F000E056F000E066F000E076F2FEC1A
:105F700030F01CC104F11DC105F11EC106F11FC1A5
:105F800007F103EC30F06A0E046F2A0E056F000E65
:105F9000066F000E076FFEEC2FF01200BF0EFA6EB8
:105FA000200E3A6F396BD89000370137023703372C
:105FB000D8B0DFEF2FF03A2FD4EF2FF039073A07A0
:105FC0000353D8B412000331070B80093F6F033924
:105FD0000F0B010F396F80EC5FF0406F390580ECDB
:105FE0005FF0405D405F396B3F33D8B039273933BC
:105FF0003FA9F4EF2FF0405139271200010138EC8E
:1060000031F0D8B01200010103510719346FFBECD5
:1060100030F0D8900751031934AF800F12000101FE
:10602000346B1FEC31F0D8A035EC31F0D8B0120051
:106030000AEC31F013EC31F01F0E366F4BEC31F0FF
:106040000B35D8B0FBEC30F0D8A00335D8B0120037
:10605000362F1EEF30F034B122EC31F01200010186
:10606000346B04510511061107110008D8A01FEC6C
:1060700031F0D8A035EC31F0D8B01200086B096BC4
:106080000A6B0B6B4BEC31F01F0E366F4BEC31F0A3
:1060900007510B5DD8A459EF30F006510A5DD8A422
:1060A00059EF30F00551095DD8A459EF30F0045193
:1060B000085DD8A06CEF30F00451085F0551D8A0FE
:1060C000053D095F0651D8A0063D0A5F0751D8A0DB
:1060D000073D0B5FD8900081362F46EF30F034B18A
:1060E00022EC31F0346B1FEC31F0D8904FEC31F0F2
:1060F00007510B5DD8A489EF30F006510A5DD8A492
:1061000089EF30F00551095DD8A489EF30F00451D2
:10611000085DD8A098EF30F0003F98EF30F0013FD5
:1061200098EF30F0023F98EF30F0032BD8B4120014
:1061300034B122EC31F012000101346B1FEC31F06C
:10614000D8B0120054EC31F0200E366F0037013712
:106150000237033711EE33F00A0E376FE7360A0EB7
:10616000E75CD8B0E76EE552372FAEEF30F0362F50
:10617000A6EF30F034B12981D890120054EC31F000
:10618000200E366F003701370237033711EE33F038
:106190000A0E376FE7360A0EE75CD8B0E76EE552B5
:1061A000372FCAEF30F0362FC2EF30F0D890120000
:1061B00001010A0E346F200E366F11EE29F03451B2
:1061C000376F0A0ED890E652D8B0E726E732372F5D
:1061D000E3EF30F00333023301330033362FDDEFCA
:1061E00030F0E750FF0FD8A00335D8B0120029B126
:1061F00022EC31F01200045100270551D8B0053DC2
:1062000001270651D8B0063D02270751D8B0073DF7
:10621000032712000051086F0151096F02510A6FE4
:1062200003510B6F12000101006B016B026B036BDA
:1062300012000101046B056B066B076B120003353E
:10624000D8A012000351800B001F011F021F031F63
:10625000003F32EF31F0013F32EF31F0023F32EFD9
:1062600031F0032B342B032512000735D8A0120080
:106270000751800B041F051F061F071F043F48EF2F
:1062800031F0053F48EF31F0063F48EF31F0072B82
:10629000342B072512000037013702370337083740
:1062A00009370A370B3712000101296B2A6B2B6B58
:1062B0002C6B2D6B2E6B2F6B306B316B326B336B0A
:1062C000120001012A510F0B2A6F2B510F0B2B6F5C
:1062D0002C510F0B2C6F2D510F0B2D6F2E510F0BBF
:1062E0002E6F2F510F0B2F6F30510F0B306F31511D
:1062F0000F0B316F32510F0B326F33510F0B336F66
:10630000120000C124F101C125F102C126F103C12F
:1063100027F104C100F105C101F106C102F107C175
:1063200003F124C104F125C105F126C106F127C1FD
:1063300007F1120010A806D08994000EC76E220E35
:10634000C66E05D08984000EC76E220EC66E050E7D
:10635000E82EFED7120010A802D0898401D08994BB
:10636000050EE82EFED712009AEC31F09E96C69EDE
:10637000000EC96EFF0E9EB602D0E82EFCD79E9688
:10638000C69E000EC96EFF0E9EB602D0E82EFCD748
:10639000C9CFAFF59E96C69E000EC96EFF0E9EB683
:1063A00002D0E82EFCD7C9CFB0F59E96C69E000E4F
:1063B000C96EFF0E9EB602D0E82EFCD7C9CFB1F54C
:1063C0009E96C69E000EC96EFF0E9EB602D0E82EA7
:1063D000FCD7C9CFB2F59E96C69E000EC96EFF0EC1
:1063E0009EB602D0E82EFCD7C9CFB3F59E96C69EC6
:1063F000000EC96EFF0E9EB602D0E82EFCD7C9CFA4
:10640000B4F59E96C69E000EC96EFF0E9EB602D0D3
:10641000E82EFCD7C9CFB5F5ABEC31F012009AEC01
:1064200031F09E96C69E800EC96EFF0E9EB602D0BB
:10643000E82EFCD79E96C69EAFC5C9FFFF0E9EB63E
:1064400002D0E82EFCD79E96C69EB0C5C9FFFF0EAF
:106450009EB602D0E82EFCD79E96C69EB1C5C9FF57
:10646000FF0E9EB602D0E82EFCD79E96C69EB2C501
:10647000C9FFFF0E9EB602D0E82EFCD79E96C69EA0
:10648000B3C5C9FFFF0E9EB602D0E82EFCD79E967C
:10649000C69EB4C5C9FFFF0E9EB602D0E82EFCD73B
:1064A0009E96C69EB5C5C9FFFF0E9EB602D0E82EC9
:1064B000FCD7ABEC31F012009AEC31F09E96C69E00
:1064C000070EC96EFF0E9EB602D0E82EFCD79E9630
:1064D000C69E000EC96EFF0E9EB602D0E82EFCD7F7
:1064E000C9CFAFF59E96C69E000EC96EFF0E9EB632
:1064F00002D0E82EFCD7C9CFB0F59E96C69E000EFE
:10650000C96EFF0E9EB602D0E82EFCD7C9CFB1F5FA
:106510009E96C69E000EC96EFF0E9EB602D0E82E55
:10652000FCD7C9CFB2F5ABEC31F09AEC31F09E96C6
:10653000C69E25C0C9FFFF0E9EB602D0E82EFCD72E
:106540009E96C69E000EC96EFF0E9EB602D0E82E25
:10655000FCD7C9CFB6F5ABEC31F012009AEC31F0B4
:106560009E96C69E870EC96EFF0E9EB602D0E82E7E
:10657000FCD79E96C69EAFC5C9FFFF0E9EB602D041
:10658000E82EFCD79E96C69EB0C5C9FFFF0E9EB6EC
:1065900002D0E82EFCD79E96C69EB1C5C9FFFF0E5D
:1065A0009EB602D0E82EFCD79E96C69EB2C5C9FF05
:1065B000FF0E9EB602D0E82EFCD7ABEC31F09AEC81
:1065C00031F09E96C69E26C0C9FFFF0E9EB602D031
:1065D000E82EFCD79E96C69EB6C5C9FFFF0E9EB696
:1065E00002D0E82EFCD7ABEC31F012009AEC31F07F
:1065F0009E96C69E870EC96EFF0E9EB602D0E82EEE
:10660000FCD79E96C69E000EC96EFF0E9EB602D0A7
:10661000E82EFCD79E96C69E800EC96EFF0E9EB6D3
:1066200002D0E82EFCD79E96C69E800EC96EFF0E45
:106630009EB602D0E82EFCD79E96C69E800EC96EEE
:10664000FF0E9EB602D0E82EFCD7ABEC31F0120064
:106650009AEC31F09E96C69E870EC96EFF0E9EB6CE
:1066600002D0E82EFCD79E96C69E000EC96EFF0E85
:106670009EB602D0E82EFCD79E96C69E000EC96E2E
:10668000FF0E9EB602D0E82EFCD79E96C69E800EC8
:10669000C96EFF0E9EB602D0E82EFCD79E96C69E0F
:1066A000800EC96EFF0E9EB602D0E82EFCD7ABEC72
:1066B00031F0120010A817D09AEC31F09E96C69EC9
:1066C0008F0EC96EFF0E9EB602D0E82EFCD79E96A6
:1066D000C69E000EC96EFF0E9EB602D0E82EFCD7F5
:1066E000ABEC31F012005CEC32F0120010A82DD0AF
:1066F0009AEC31F09E96C69E26C0C9FFFF0E9EB64C
:1067000002D0E82EFCD79E96C69E450EC96EFF0E9F
:106710009EB602D0E82EFCD7ABEC31F09AEC31F00B
:106720009E96C69E8F0EC96EFF0E9EB602D0E82EB4
:10673000FCD79E96C69E000EC96EFF0E9EB602D076
:10674000E82EFCD7ABEC31F012009AEC31F09E96BB
:10675000C69E26C0C9FFFF0E9EB602D0E82EFCD70B
:106760009E96C69E010EC96EFF0E9EB602D0E82E02
:10677000FCD7ABEC31F09AEC31F09E96C69E910EB0
:10678000C96EFF0E9EB602D0E82EFCD79E96C69E1E
:10679000A50EC96EFF0E9EB602D0E82EFCD7ABEC5C
:1067A00031F012009AEC31F09E96C69E26C0C9FFC9
:1067B000FF0E9EB602D0E82EFCD79E96C69E810E96
:1067C000C96EFF0E9EB602D0E82EFCD7ABEC31F0BE
:1067D00012009AEC31F09E96C69E26C0C9FFFF0EAD
:1067E0009EB602D0E82EFCD79E96C69E010EC96EBC
:1067F000FF0E9EB602D0E82EFCD7ABEC31F01200B3
:106800009AEC31F09E96C69E910EC96EFF0E9EB612
:1068100002D0E82EFCD79E96C69EA50EC96EFF0E2E
:106820009EB602D0E82EFCD7ABEC31F012009AEC09
:1068300031F09E96C69E910EC96EFF0E9EB602D096
:10684000E82EFCD79E96C69E000EC96EFF0E9EB621
:1068500002D0E82EFCD7ABEC31F012000501256B1D
:10686000266B276B286B899A400EC76E200EC66E6A
:106870009E96C69E030EC96EFF0E9EB602D0E82EEF
:10688000FCD79E96C69E27C5C9FFFF0E9EB602D0B6
:10689000E82EFCD79E96C69E26C5C9FFFF0E9EB663
:1068A00002D0E82EFCD79E96C69E25C5C9FFFF0ED6
:1068B0009EB602D0E82EFCD79E96C69EC952FF0E09
:1068C0009EB602D0E82EFCD7898A0F01C950FF0A74
:1068D00001E1120005012E51130A05E005012E51B8
:1068E000170A0CE012000501E00E256FFF0E266F5F
:1068F0000F0E276F000E286F87EF34F00501E00EB2
:10690000256FFF0E266FFF0E276F000E286F899AE6
:10691000400EC76E200EC66E9E96C69E030EC96EB2
:10692000FF0E9EB602D0E82EFCD79E96C69E27C5C7
:10693000C9FFFF0E9EB602D0E82EFCD79E96C69EDB
:1069400026C5C9FFFF0E9EB602D0E82EFCD79E9644
:10695000C69E25C5C9FFFF0E9EB602D0E82EFCD705
:106960009E96C69EC952FF0E9EB602D0E82EFCD758
:10697000898A0F01C950FF0A1DE005012E51130A33
:1069800005E005012E51170A0BE012000501000E6B
:10699000256F000E266F100E276F000E286F120055
:1069A0000501000E256F000E266F000E276F010EE9
:1069B000286F12000501256B266B276B286B0501DC
:1069C0002E51130A05E005012E51170A0CE01200A2
:1069D0000501000E216F000E226F080E236F000EBE
:1069E000246FFCEF34F00501000E216F000E226FC2
:1069F000800E236F000E246F21C500F122C501F126
:106A000023C502F124C503F125C504F126C505F10E
:106A100027C506F128C507F14FEC2EF000C125F57A
:106A200001C126F502C127F503C128F5899A400E58
:106A3000C76E200EC66E9E96C69E030EC96EFF0ED2
:106A40009EB602D0E82EFCD79E96C69E27C5C9FFEB
:106A5000FF0E9EB602D0E82EFCD79E96C69E26C597
:106A6000C9FFFF0E9EB602D0E82EFCD79E96C69EAA
:106A700025C5C9FFFF0E9EB602D0E82EFCD79E9614
:106A8000C69EC952FF0E9EB602D0E82EFCD7898A58
:106A9000C950FF0A08E104C125F505C126F506C164
:106AA00027F507C128F5D890050124332333223375
:106AB00021332151E00B216F0501216767EF35F08C
:106AC000226767EF35F0236767EF35F02467FCEF47
:106AD00034F00501200E2527E86A2623E86A2723DB
:106AE000E86A28231200E86A05012E51130A06E01D
:106AF00005012E51170A0BE0020E12000501285164
:106B0000000A03E12751F00B07E0010E1200050116
:106B10002851000A01E0010E120029C500F12AC522
:106B200001F12BC502F12CC503F125C504F126C5E1
:106B300005F127C506F128C507F1FEEC2FF003BFCC
:106B4000120073EC35F0D8A405EF36F0899A400EA8
:106B5000C76E200EC66E9E96C69E060EC96EFF0EAE
:106B60009EB602D0E82EFCD7898A899A9E96C69E48
:106B7000020EC96EFF0E9EB602D0E82EFCD79E967E
:106B8000C69E27C5C9FFFF0E9EB602D0E82EFCD7D1
:106B90009E96C69E26C5C9FFFF0E9EB602D0E82E61
:106BA000FCD79E96C69E25C5C9FFFF0E9EB602D095
:106BB000E82EFCD79E96C69E000EC96EFF0E9EB6AE
:106BC00002D0E82EFCD7898A899A9E96C69E050E29
:106BD000C96EFF0E9EB602D0E82EFCD79E96C69ECA
:106BE000C952FF0E9EB602D0E82EFCD7C9B0EEEF18
:106BF00035F0898A0501200E2527E86A2623E86AF0
:106C00002723E86A28238DEF35F01200899A400E79
:106C1000C76E200EC66E9E96C69E060EC96EFF0EED
:106C20009EB602D0E82EFCD7898A899A9E96C69E87
:106C3000C70EC96EFF0E9EB602D0E82EFCD7898A19
:106C40000501256B266B276B286B1200899A400E75
:106C5000C76E200EC66E9E96C69E050EC96EFF0EAE
:106C60009EB602D0E82EFCD79E96C69EC952FF0E55
:106C70009EB602D0E82EFCD7C9CF37F5898A12001C
:106C8000899A400EC76E200EC66E9E96C69EB90E9D
:106C9000C96EFF0E9EB602D0E82EFCD7898A12007C
:106CA000899A400EC76E200EC66E9E96C69EAB0E8B
:106CB000C96EFF0E9EB602D0E82EFCD7898AFF0E61
:106CC000E82EFED7120073EC35F0D8A41200899A92
:106CD000400EC76E200EC66E9E96C69E030EC96EEF
:106CE000FF0E9EB602D0E82EFCD79E96C69E27C504
:106CF000C9FFFF0E9EB602D0E82EFCD79E96C69E18
:106D000026C5C9FFFF0E9EB602D0E82EFCD79E9680
:106D1000C69E25C5C9FFFF0E9EB602D0E82EFCD741
:106D20009E96C69EC952FF0E9EB602D0E82EFCD794
:106D3000898A0F01C950FF0AD8A4E2EF37F0050194
:106D4000FE0E376F0501FF0E536FFF0E546FFF0EDF
:106D5000556FFF0E566F15A637991586B4EC31F0B6
:106D6000AFC538F5B0C539F5B1C53AF5B2C53BF593
:106D7000B3C53CF5B4C53DF5B5C53EF50784BAC10C
:106D800066F1BBC167F1BCC168F1BDC169F14BC11E
:106D90004FF14CC150F14DC151F14EC152F157C1AB
:106DA00059F158C15AF100011650010AD8B4E7EF61
:106DB00036F000011650020AD8B40CEF37F000018B
:106DC0001650040AD8B431EF37F0E2EF37F005017E
:106DD000476B486B496B4A6B05014B6B4C6B4D6BBA
:106DE0004E6B05014F6B506B516B526B8BA0379BF9
:106DF000EAEC22F000C1DAF101C1DBF102C1DCF101
:106E000003C1DDF100C13FF501C140F502C141F50B
:106E100003C142F550EF37F00501476B486B496BF2
:106E20004A6B05014B6B4C6B4D6B4E6B05014F6B09
:106E3000506B516B526BEAEC22F000C1DAF101C1E8
:106E4000DBF102C1DCF103C1DDF1E7EC23F000C1AD
:106E500047F501C148F502C149F503C14AF5E2EF22
:106E600037F0379BDAC13FF5DBC140F5DCC141F5B6
:106E7000DDC142F5EAEC22F000C14BF501C14CF551
:106E800002C14DF503C14EF5E7EC23F000C14FF50B
:106E900001C150F502C151F503C152F550EF37F071
:106EA000050161675BEF37F062675BEF37F063679F
:106EB0005BEF37F064675FEF37F074EF37F0DAC1FC
:106EC00000F1DBC101F1DCC102F1DDC103F161C5FB
:106ED00004F162C505F163C506F164C507F1FEEC76
:106EE0002FF003BFE2EF37F059C143F55AC144F523
:106EF000B9C545F50501210E326F899A400EC76E5E
:106F0000200EC66E9E96C69E060EC96EFF0E9EB6DB
:106F100002D0E82EFCD7898A899A9E96C69E020ED8
:106F2000C96EFF0E9EB602D0E82EFCD79E96C69E76
:106F300027C5C9FFFF0E9EB602D0E82EFCD79E964D
:106F4000C69E26C5C9FFFF0E9EB602D0E82EFCD70E
:106F50009E96C69E25C5C9FFFF0E9EB602D0E82E9E
:106F6000FCD725EE37F0322F02D0C2EF37F09E96D5
:106F7000C69EDECFC9FFFF0E9EB602D0E82EFCD71C
:106F8000B3EF37F0898A899A9E96C69E050EC96E20
:106F9000FF0E9EB602D0E82EFCD79E96C69EC95222
:106FA000FF0E9EB602D0E82EFCD7C9B0CDEF37F069
:106FB000898A0501200E2527E86A2623E86A272307
:106FC000E86A282315900794120021C500F122C514
:106FD00001F123C502F124C503F1899A400EC76E61
:106FE000200EC66E9E96C69E0B0EC96EFF0E9EB6F6
:106FF00002D0E82EFCD79E96C69E02C1C9FFFF0EA6
:107000009EB602D0E82EFCD79E96C69E01C1C9FF4F
:10701000FF0E9EB602D0E82EFCD79E96C69E00C1FB
:10702000C9FFFF0E9EB602D0E82EFCD79E96C69EE4
:10703000C952FF0E9EB602D0E82EFCD725EE37F0DF
:107040000501200E326F9E96C69EC952FF0E9EB657
:1070500002D0E82EFCD7C9CFDEFF322F23EF38F065
:10706000898A1200899A400EC76E200EC66E9E96BF
:10707000C69E900EC96EFF0E9EB602D0E82EFCD7BB
:107080009E96C69E000EC96EFF0E9EB602D0E82EDA
:10709000FCD79E96C69E000EC96EFF0E9EB602D00D
:1070A000E82EFCD79E96C69E000EC96EFF0E9EB6B9
:1070B00002D0E82EFCD79E96C69EC952FF0E9EB601
:1070C00002D0E82EFCD7C9CF2DF59E96C69EC95298
:1070D000FF0E9EB602D0E82EFCD7C9CF2EF5898AC6
:1070E0001200B4EC31F005012F51010A5FE00501F7
:1070F0002F51020A16E005012F51030A19E005017C
:107100002F51040A24E005012F51050A2BE0050147
:107110002F51060A39E005012F51070A3FE0D6EF4B
:1071200038F0602FD4EF38F05FC560F5D6EF38F057
:10713000B0C500F101010F0E001701010051000A56
:1071400035E001010051050A31E0D4EF38F0B0C557
:1071500000F101010F0E001701010051000A26E0A5
:10716000D4EF38F00501B051000A20E00501B0511C
:10717000150A1CE00501B051300A18E00501B051B4
:10718000450A14E0D4EF38F00501B051000A0EE0D2
:107190000501B051300A0AE0D4EF38F00501B051D2
:1071A000000A04E0D4EF38F01590120015801200A8
:1071B0008B90CAEC2EF0B9C5E8FFD70802E3CAEC01
:1071C0002EF0B9C5E8FFC80802E3CAEC2EF0B9C535
:1071D000E8FFB90802E3CAEC2EF0B9C5E8FFAA0837
:1071E00002E3CAEC2EF0B9C5E8FF9B0802E3CAEC43
:1071F0002EF040EC36F0F29CF29E8B94C69AC29030
:107200009482948C720ED36ED3A4FED789968A9002
:107210009390F29AF2949D909E909D929E92F298F5
:10722000F2925AEC33F0FF0EE8CF00F0E82EFED7D2
:10723000002EFCD7F290F286815081A822EF39F01F
:10724000F29E0300700ED36EF296F29015840380C6
:08725000EBEC2EF09AEF0BF0BD
:10BF0000E844F926000C160C2B0C3F0C520C640C68
:10BF1000760C860C960CA50CB30CC10CCF0CDC0C6B
:06BF2000E80CF40C000C1B
:0200000400F00A
:0100C800FE39
:00000001FF
